:020000040000FA
:1000000004000400AFEF0EF0086A800E396E39D09C
:10001000186A196A0A9A79EC02F0D8A01200D30F74
:10002000D8B40A8A2D0FC60F03E20A0FF4E305D0F5
:10003000F30FF1E2060FEFE30A0F146E040E156ED4
:10004000D89018361936152EFBD7145018120806FA
:100050000FE079EC02F0D8A01200C60F03E20A0FFD
:1000600007E3EBD7F30F04E2060F02E30A0FE5D72D
:100070000AAA04D0181E191E184A192A1850D88026
:100080001200186A196A1A6A1B6A0A9A79EC02F055
:10009000D8A01200D30FD8B40A8A2D0FC60FF6E2EB
:1000A0000A0FF4E3146E136A126A116A0A0E106ED4
:1000B0005AEC04F014501024186E1150196E000EF2
:1000C000D8B0010E192612501A6E000ED8B0010ECB
:1000D0001A2613501B6E000ED8B0010E1B26080600
:1000E00008E079EC02F0D8A01200C60F02E20A0F75
:1000F000D9E20AAA0BD0181E191E1A1E1B1E182A96
:10010000D8B4192AD8B41A2AD8B41B2A1850D880BF
:100110001200086A186E196A00960850D8B4008652
:10012000040E076E193805D8195003D8183801D8AD
:1001300018500F0BF60FD8B0070F0A0F28D0086A17
:10014000186E196A18BE196832D803D0086A186E7A
:10015000196A00960850D8B40086050E076E270E5F
:10016000156E100E0CD8030E156EE80E08D8156A21
:10017000640E05D8156A0A0E02D8185008D0146EFD
:100180001950116E1850106E43EC04F01050106EA0
:10019000074E0096085003E0075CD8B007D0105017
:1001A000D8A4009600B602D0300F93D1120019AE39
:1001B000120018501910D8B41200181E191E184A2F
:1001C000192A2D0E86D13B6E24AE02D02D0E81D978
:1001D000263E04D0253E02D0244A242A316A326ABF
:1001E000336A346A248E6A0E2326D890243225324C
:1001F00026323432333232323132233EF6D7265071
:10020000235C2626235E2550245C2526245E086A6E
:1002100039D82E0E5ED93C6AD8903134266E3234ED
:10022000256E3334246E3434236E3C36D890263613
:100230002536243623363C36315026263250D8B067
:10024000323C25263350D8B0333C24263450D8B025
:10025000343C2326D8B03C3ED8902636253624366A
:1002600023363C363C50300F34D926C031F025C0FF
:1002700032F024C033F023C034F03B2ECCD7D890DA
:10028000120028D80096085003E100860A0E086E76
:1002900026C013F025C012F024C011F023C010F0C6
:1002A000076A1B6A1A6A196A0A0E186E15EC04F0BE
:1002B000072A0750085CD8A4F4D71850D8A4009691
:1002C00000A602D0082C03D01850300F02D9082EF7
:1002D000DFD7120026AE1200D880000E2356245617
:1002E000255626562D0EF5D0186E0750D8B412009C
:1002F00018C0E9FF19C0EAFFEF50D8B41200E9D8DE
:10030000184A192A0706F1D705C010F006C011F0E7
:10031000010E146E156AEA6802C0E9FF04002AD8CB
:10032000D8A015D0142EFAD7FF0E1526D8B0F6D7C0
:100330001026D8A01126D8A01200320E146E156A0D
:10034000EDD7EA6802C0E9FF040014D8FDE254D8F2
:100350001E6A080E156E51D80DD8D8B01E3E143244
:10036000152EF9D720AA1E6A20BA149E46D8D88026
:1003700014501200120EE9260950EF1202C0E9FFD4
:10038000EF1420BC0918FF0F12001C6EEA68E26827
:100390000250E96E120FE16E800E0A16080E1D6EF5
:1003A000D890D8B00A3E11D81C321D2EFAD70400BE
:1003B00020BA0A300AD800D000D000D0D88005D8A2
:1003C0000650156E055092D9120020AE0BD0EF509A
:1003D000091020AC0918EF6EE7500910D8A00918D1
:1003E000E76E0BD0EF500910D8A0091820BC0918EF
:1003F000EF6E091CE71601D00A8C20501F0BFF0F6F
:10040000116E1F50F70FD8B0112A0AAC7CD10A9C8C
:10041000106E020EACEC04F076D1ABB2AB98AB88A8
:1004200002C010F009C011F0146A156A040000D06F
:1004300004009EBA14D0E868142615221022112256
:10044000D8A012001448153CF1D73D0E146E156A61
:10045000EFD7ABB2AB98AB8804009EAAFED7AE50E4
:10046000D880120004009EA8FED7AD6E120071B2B3
:100470007198718802C010F009C011F0146A156AF1
:10048000040000D00400A4BA14D0E8681426152291
:1004900010221122D8A012001448153CF1D73D0EAD
:1004A000146E156AEFD771B2719871880400A4AA0E
:1004B000FED77450D8801200A66AA68E0900F550A7
:1004C00002E002D8FBD712000400A4A8FED7736E86
:1004D000120001BA5AD701B4C5D701A202D001B0A7
:1004E0003CD001A205D001B003D001B2EE6E1200E3
:1004F000EBD7395292E03904ACE03950080AB7E042
:100500003950090AD0E03950030AD8B4FDD6395021
:10051000050AD8B416D7D88039BEEE50120000882C
:1005200000A8009800BA03D0008A35D829E20094C8
:10053000080E156E40D81436152EFCD700B407D01F
:1005400000B801D04AD845D841D800B819D843D806
:10055000D89014501CD0008800A8009800BC05D08A
:10056000FE0B0A6E008CD89012D000BE05D01C6E17
:10057000008E11D805E21C5012D802E200A807D064
:100580002CD827D8009C009E009A009424D81E8066
:10059000D8A01E90120017D80A5000BA0109146E94
:1005A000080E156E143617D801E217D812D80ED8D7
:1005B000152EF8D710D80DD800D00400D89081BCE3
:1005C000D88004D8120007D804D807D8819E939EFB
:1005D00006D0938E04D0938C02D08A9C939C1200F8
:1005E000AA6AA96EA66AA680A850A94AAA2A1200D9
:1005F000AA6AA86EA66AA684550EA76EAA0EA76E52
:10060000A6820400A6B2FED7A694A94AAA2A12007E
:10061000E836E836FC0B0109C2128009C216C05048
:10062000F80B0309C06E640E6DD8C2820400C2B21A
:10063000FED7C4CF24F0C350236E1200080E1C6EE8
:100640001D6EEA6803C0E9FF04500AB489D90AA400
:1006500089D9E26803C0E1FFEA6802C0E9FF0950F6
:10066000E988E92AEC1202C0E9FF106A116A1C50FD
:10067000D8B412000AB234D8EF500914FF0F103664
:1006800011360AA22DD81C2EF5D71D500AB053D111
:1006900010501200080E1C6EEA6803C0E9FF0450F7
:1006A0000AB45ED90AA45ED9E26803C0E1FFEA6831
:1006B00002C0E9FF091CE988E92AEC161C50D8B4ED
:1006C00012000AB038D902C0E9FF11321032EF50DF
:1006D0000910D8A00918EF6E03D81C2EF6D7120007
:1006E0000450E71A0400E71A1200156A146EFF0E90
:1006F0001426152200D0D8A01200030E116EDE0EB3
:1007000002D8F5D7116AE90F106EFC0E05E304005C
:1007100004001026FDE2040010261106F9E210B0D4
:1007200000D010A202D000D0040012000009D8B4FA
:1007300012001E6E10C0E9FF11C0EAFF116A106AB4
:100740001EBE07D0EE50106E1EA21200EF50116EAA
:10075000120004D8EF14D8A4102A1200010E1EB003
:10076000E8441EB2E8441EB2E8441EB4E838120061
:1007700013501B18800BF46E13AE06D0D880000EF9
:1007800010561156125613561BAE06D0D880000EC6
:10079000185619561A561B56146A156A166A176A9D
:1007A0002D6A2E6A2F6A306A1B501A101910181001
:1007B00023E0200EF36ED890103611361236133621
:1007C0002D362E362F36303618502D5C19502E58B7
:1007D0001A502F581B50305809E318502D5E1950ED
:1007E0002E5A1A502F5A1B50305AD88014361536AC
:1007F00016361736F32EDFD7F4AE06D0D880000EAB
:10080000145615561656175614C010F015C011F090
:1008100016C012F017C013F02DC018F02EC019F03A
:100820002FC01AF030C01BF012002D6A2E6A2F6AFA
:10083000306A210E166E15D02D362E362F363036F4
:1008400018502D5C19502E581A502F581B503058E4
:1008500008E3306E18502D5E19502E5A1A502F5A38
:10086000D8801036113612361336162EE5D730C022
:100870001BF02FC01AF02EC019F02D50186E120068
:10088000116A156A146E196A186A100EF36E113423
:10089000183619361450185C1550195805E31450C1
:1008A000185E1550195AD88010361136F32EEFD72E
:1008B0001050120013C030F012C02FF011C02EF0F3
:1008C00010C02DF02F501802F3CF12F0F4CF13F018
:1008D0002E501902F3501226F45013222D501A02F2
:1008E000F3501226F450132230501802F3501326FE
:1008F0002F501902F35013262E501A02F3501326CC
:100900002D501B02F35013262D501802F3CF10F078
:10091000F4CF11F02E501802F3501126F450122289
:10092000000E13222D501902F3501126F4501222FA
:10093000000E13221200146A156A04D0113210320C
:1009400014361536FF0FFAE215C011F01450106E70
:100950001200D89011321032FF0FFBE2105012003B
:10096000EF1203D0FF0AEF1601D0FF0AE988E92A47
:10097000EC161200A66AA68E0900F55002E0EE6E93
:10098000FBD71200A66AA68EEE500900F55C02E1C4
:10099000F566FAD712003DC01EF03D8C0ED8D90E78
:1009A000386E5B0E376E5E0E366E7D0E356E9BECCE
:1009B00007F01EAC3D9C3450120032BE09D13152BA
:1009C000D8B406D13DC01CF03D8C7E0E315C1D6E4E
:1009D0007E0E316E386A376A366A7F0E356EF30ED8
:1009E000345C040ED8A0050E335C350ED8A0360E4C
:1009F000325C02E3AAD903D0312AA7D91D0634C03C
:100A000010F033C011F032C012F031C013F0710E8B
:100A1000386E5F0E376E550E366E800E356E97D976
:100A200010C038F011C037F012C036F013C035F0E6
:100A30009BEC07F0C60E386EF50E376E1F0E366E45
:100A4000800E356E84D934C014F033C015F032C036
:100A500016F031C017F010C034F011C033F012C0DE
:100A600032F013C031F08A0E386E120E376E790EE6
:100A7000366E7D0E356E9BEC07F0F60E386E460E28
:100A8000376E550E366E7E0E356E61D914C038F055
:100A900015C037F016C036F017C035F0E6D934C0AF
:100AA00014F033C015F032C016F031C017F01350F7
:100AB000316E356E1250326E366E1150336E376EA7
:100AC0001050346E386E9BEC07F034C023F033C006
:100AD00024F032C025F031C026F014C038F015C023
:100AE00037F016C036F017C035F09BEC07F010C099
:100AF00038F011C037F012C036F013C035F09BEC5F
:100B000007F023C038F024C037F025C036F026C0E7
:100B100035F03566350619D910C038F011C037F0F8
:100B200012C036F013C035F012D91D5252E034C055
:100B300023F033C024F032C025F031C026F01DC0B0
:100B400031F0000E31BEFF0E326E336E346E48EC63
:100B500008F034C010F033C011F032C012F031C0D0
:100B600013F0830E386E800E376EDE0E366E720E08
:100B7000356EE1D923C038F024C037F025C036F0F7
:100B800026C035F0E4D834C023F033C024F032C09E
:100B900025F031C026F010C034F011C033F012C07F
:100BA00032F013C031F0386A800E376E310E366E77
:100BB0007E0E356EC0D923C038F024C037F025C072
:100BC00036F026C035F0C3D81CBC03D03D9C01D004
:100BD0003D8A34501200365032183F6E3FBE30D03E
:100BE00036BE17D03550315CD8A0000CD8A4010C0B
:100BF0003650325CD8A0000CD8A4010C3750335CBE
:100C0000D8A0000CD8A4010C3850345CD8A0000C3B
:100C1000010C3150355CD8A0000CD8A4010C325026
:100C2000365CD8A0000CD8A4010C3350375CD8A097
:100C3000000CD8A4010C3450385CD8A0000C010C76
:100C400032AE010C000C365032183F6E3FBE34D02D
:100C500036BE19D03550315CD8A0000CD8A4010C98
:100C60003650325CD8A0000CD8A4010C3750335C4D
:100C7000D8A0000CD8A4010C3850345CD8A0000CCB
:100C8000D8A4010C000C3150355CD8A0000CD8A4BD
:100C9000010C3250365CD8A0000CD8A4010C3350A3
:100CA000375CD8A0000CD8A4010C3450385CD8A014
:100CB000000CD8A4010C000C32AE010C000C325018
:100CC00036183F6E3FBE34D032BE19D03150355C3D
:100CD000D8A0000CD8A4010C3250365CD8A0000C6F
:100CE000D8A4010C3350375CD8A0000CD8A4010C58
:100CF0003450385CD8A0000CD8A4010C000C35503E
:100D0000315CD8A0000CD8A4010C3650325CD8A0BD
:100D1000000CD8A4010C3750335CD8A0000CD8A428
:100D2000010C3850345CD8A0000CD8A4010C000C85
:100D300036AE010C000C386A376A7E0E356E800EB6
:100D400032AE000E366E03D844D1800E361A3550BE
:100D5000315C3C6E11E23C6C315035C031F0356E87
:100D6000325036C032F0366E335037C033F0376E03
:100D7000345038C034F0386E1A0E3C6074D035529E
:100D800072E03B6A32503E6E3618406E328E368EBE
:100D9000080E3C5E08E338C03BF037C038F036C080
:100DA00037F0366AF5D73C2607E0D890363237322E
:100DB00038323B323C2EF9D740AE33D03850345E17
:100DC0003750335A3650325A07E2D880000E345624
:100DD00033563256800E3E1A3B6C04E03406000E49
:100DE000335A325A040E3C6E32660DD033C032F0A4
:100DF00034C033F03BC034F03B6A080E315E29E367
:100E00003C2EF2D726D032BE08D0D8903B363436AE
:100E100033363236312EF7D71CD03BAE22D03B6A68
:100E20000FD038503426375033223650322206E362
:100E30003232333234323B32314A0DD03BAE11D0F4
:100E4000343E0FD0333E0DD0323E0BD0D88034909C
:100E5000EFD7316A02D03D823168346A336A800E3E
:100E6000326E3EAE329E3450120032502F6E361823
:100E7000406E355051E0315252E0315E7F0E03E258
:100E8000312603E24BD031264CE234C02DF033C082
:100E90002EF02F8E368E180E3E6E346A336A326A0A
:100EA0000BD038502D5C37502E5811E32E6E2F6A20
:100EB00038502D5E0BD004E236502F5CF2E007E391
:100EC00038502D5E37502E5A36502F5AD88034362F
:100ED000333632362D362E362F363E2EECD732BEF6
:100EE00007D031521BE0403231063E2A4036E3D76C
:100EF00007E238502D5E37502E5A36502F5A17E3DE
:100F0000343E15D0333E13D0323E11D0323233321C
:100F10003432313E0CD005D03D8604D03D84316A58
:100F200002D03D823168346A336A800E326E40AE40
:100F3000329E3450120032502F6E3618406E3150AF
:100F4000D8A435503AE031267E0E03E3315E03E348
:100F500036D0315E31E334C02DF033C02EF02F8E09
:100F6000368E346A336A326A180E3E6E2F322E3253
:100F70002D3206E338503426375033223650322291
:100F80003232333234323E2EF1D732BE07D03436CD
:100F900033363236315210E031062F3416E3343E08
:100FA00014D0333E12D0323E10D0D8803232333299
:100FB0003432313E0AD003D03D84316A02D03D82C2
:100FC0003168346A336A800E326E40AE329E3450DD
:100FD000120031C03EF0325034C032F0346E34363C
:100FE0003E3234323D6A34363E3602E33D843D7E45
:100FF00006E13D803E6A346A336A326A0BD03E288D
:1010000003E0D880343206D0D890343202E13D82F9
:1010100001D03D863DB604D03DA20FD03DB407D0EF
:101020007F0E346EFF0E336E326E316E23D0800E23
:10103000346E01D0346A000EF6D73DB0FBD7316A6A
:101040009F0E3E60EBD77E0E3E64F4D79E0E3E5C54
:1010500007E0D89034323332323231323E2AF6D77A
:101060003DA408D0D880000E31563256335634563F
:1010700034AEE0D731501200000E32BEFF0E336E98
:10108000346E06D0316E326A336A346A409E0AD0BA
:10109000409E34AE07D0D880000E315632563356BB
:1010A0003456408E960E3E6E345209E0080E3E26AF
:1010B00032C031F033C032F034C033F011D033528B
:1010C0000FE1080E3E5E325007E1080E3E5E3150E1
:1010D00002E1345010D0316A336E31C032F0316ADF
:1010E00033BE06D0D8903136323633363E06F8D786
:1010F00040AE339E3E5031C034F0316E335032C07A
:1011000033F0326E120024505542582C34302C47A4
:101110004C4C2C302C302C302C302A3543002450B1
:101120005542582C34302C5A44412C302C302C3021
:101130002C302A34340024505542582C34302C475B
:1011400053562C302C302C302C302A35390024507A
:101150005542582C34302C4753412C302C302C30F5
:101160002C302A34450024505542582C34302C520F
:101170004D432C302C302C302C302A343700245066
:101180004D544B3331342C302C302C302C312C300E
:101190002C302C302C302C302C302C302C302C306F
:1011A0002C302C302C302C302C302C302A32390082
:1011B00024505542582C34302C5654472C302C3067
:1011C0002C302C302A35450024504D544B333134CB
:1011D0002C302C302C312C312C302C302C302C302D
:1011E0002C302C302C302C302C302C302C302C301F
:1011F0002C302C302C302A32380024505542582CB8
:1012000034302C5654472C312C302C302C302A358D
:10121000460024504D544B3136312C302A323800A0
:1012200024504D544B3130322A333100244750473B
:1012300047412C3030323135332E3030302C343879
:1012400031352E393038302C4E2C30313934392E5E
:10125000323132302C452C312C31302C312E322C85
:101260003231372E302C4D2C2D33342E322C4D2C48
:101270002C303030302A3545000024475056544732
:101280002C3330392E36322C542C202C4D2C302E31
:1012900031332C4E2C302E322C4B2C412A32330041
:1012A0002020202047505320434F4D4D554E494359
:1012B0004154494F4E204552524F522020200000A9
:1012C0002020202047505320435243204552524F64
:1012D00052202020000042414C4C4F4F4E205041A4
:1012E000594C4F4144205620000045204259204F80
:1012F0004D3342430000547970652048454C5020DE
:10130000666F7220496E666F0000435749440000C3
:1013100043574300435743414C4C000043574C0054
:1013200043574C4F43004C4F4341544F52004C4F96
:101330004331300043414C4C00004652510046526C
:10134000455155454E43590044455600444556497C
:101350004154494F4E0042415544000053504545C9
:101360004400444249545300534249545300504F9F
:1013700055540000504F5745520049445350000007
:10138000435753500000534F4C41520055534F4C5C
:10139000000054454D500000494E54454D5000004A
:1013A000505245535300435742415400435754450C
:1013B0004D500000434F5552534500004241545692
:1013C000000053555056000049534F4C0000534500
:1013D0004E540000444953500000524546005443C7
:1013E000584F00004F4646534554000048454C5066
:1013F0000000444154410000534C454550005445C1
:101400005354000054554E45000053455247505325
:10141000000043414C494252415445005345545009
:1014200000004E4F4750530055424C4F5800564510
:101430005200455849540000436F6D6D616E642041
:101440006973206E6F742076616C696400005520AA
:101450002D204652512055702C2044202D204652DC
:101460005120446F776E2C2045202D2045786974DB
:10147000000055424C4F58200000534F4C415263DE
:10148000656C6C20000054454D5065726174757236
:1014900065200000494E7465726E616C54454D5074
:1014A00065726174757265200000737065656420F3
:1014B0002620434F555253452000424154566F6CED
:1014C000746167652000535550706C79566F6C7469
:1014D000616765200000536F6C6172566F6C7461B8
:1014E00067652000536F6C617243757272656E742C
:1014F000200053454E54656E6365200043574241BA
:1015000054200000435754454D5020004C4F434158
:10151000544F522000004C4F4331302000004357BD
:101520004C4F43200000534C4545502000004341A0
:101530004C4C3A200000435743414C4C3A200000A9
:101540004652455155454E43593A20004445564967
:101550004154494F4E3A200053504545443A2000EB
:101560004441544120424954533A200053544F506F
:1015700020424954533A2000504F574552204F556E
:10158000543A2000435749442073706565643A20FB
:1015900000004D4F44454D204F46465345543A2098
:1015A0000000584F204652455155454E43593A2068
:1015B0000000534552475053200034383030204209
:1015C0006400393630302042640031393230302006
:1015D000426400004F534354554E453A200056454F
:1015E0005253494F4E3A204243504C20762E000031
:1015F000564261743A20000054656D703A20000034
:10160000436F6D6D616E647320287769746820651F
:1016100078616D706C65293A200044495350202050
:10162000202D20646973706C617920616C6C20736B
:101630006574696E6773000043414C4C2020202D77
:10164000206964656E74696669657220666F7220D0
:101650007061796C6F616400435743414C4C202D9D
:10166000204357206964656E74696669657200007D
:10167000465251202020202D206672657175656EBE
:10168000637920696E20487A0000504F57455220F8
:101690006F7220504F5554202D206F7574707574E3
:1016A00020706F77657220696E2064426D0052452C
:1016B00046202020202D20584F206F722054435860
:1016C0004F206672657175656E637920696E20487A
:1016D0007A20286D696E2E20313030303030303035
:1016E0002C206D61782E2033333030303030300094
:1016F0005443584F2020202D204F4E3D5443584FE7
:101700002C204F46463D584F00004F464653455407
:10171000202D206D6F64656D206672657175656E34
:101720006379206F666673657420696E20487A203D
:10173000286D61782E202B2D333030303029000079
:10174000444556202020202D206465766961746907
:101750006F6E20696E20487A000042415544202077
:10176000202D20626175647261746520666F72203D
:1017700052545459207472616E736D697474696E39
:101780006700444249545320202D206E756D6265D8
:1017900072206F66206461746162697473005342E1
:1017A00049545320202D206E756D626572206F663E
:1017B0002073746F706269747320312E35203D2060
:1017C0003135000049445350206F72204357535025
:1017D000202D207370656564206F66204357206953
:1017E00064656E74696669657220696E2057504D34
:1017F0000000435749442020202D2073656E64204B
:101800004357206964656E746966696572204F4E3E
:10181000206F72204F464600435742415420202DEE
:101820002073656E642062617465727920766F6CD6
:101830007461676520696E204357202D204F4E202C
:101840006F72204F4646000043574C202020202D29
:101850002073656E6420515241206C6F632E2061AD
:101860006E6420616C74697475646520696E2043D0
:1018700057202D204F4E206F72204F464600434F79
:1018800055525345202D2073656E6420636F757229
:10189000736520616E64207370656564202D204F30
:1018A0004E206F72204F4646000042415456202081
:1018B000202D2073656E64206261746572792076D4
:1018C0006F6C74616765202D204F4E206F72204F22
:1018D00046460000535550562020202D2073656E3B
:1018E0006420737570706C7920766F6C74616765B5
:1018F000202D204F4E206F72204F46460000505240
:1019000045535320202D20707265737375726520C6
:1019100073656E736F72206D6F756E746564202DC4
:10192000204F4E206F72204F46460000534F4C41CF
:101930005220202D20736F6C617263656C6C206D7A
:101940006F756E746564204F4E2879657329206F1A
:1019500072204F4646286E6F290055534F4C202069
:10196000202D2073656E6420736F6C617220766F1A
:101970006C74616765202D204F4E206F72204F469A
:10198000460049534F4C2020202D2073656E642063
:10199000736F6C61722063757272656E74204F4E46
:1019A000206F72204F46460055424C4F5820202D44
:1019B000204F4E203D2055424C4F58204F46462048
:1019C0003D205155454354454C0054454D50202031
:1019D000202D2073656E6420696E626F78207465B7
:1019E0006D7065726174757265202D2059455320A4
:1019F0006F72204E4F00494E54454D50202D20739C
:101A0000656E6420726164696F63686970207465D3
:101A10006D7065726174757265202D205945532073
:101A20006F72204E4F00455854454D50202D207365
:101A3000656E642065787465726E616C2074656D86
:101A40007065726174757265202D20594553206F41
:101A500072204E4F00004C4F4341544F522D207383
:101A6000656E6420515241206C6F6361746F722007
:101A70002D204F4E206F72204F4646004C4F433171
:101A80003020202D2073656E642031302063686122
:101A9000722E206F6620515241206C6F632E204FB2
:101AA0004E203D2031302C204F4646203D20362010
:101AB00063686172616B74657273000053454E54C4
:101AC0002020202D2073656E64204F4E203D207312
:101AD000656E74656E6365202F204F4646203D205D
:101AE00076697369626C6520736174656C6974658D
:101AF0007300534C45455020202D20737769746343
:101B00006820746865204750532072656365697664
:101B10006572202D204F4E206F72204F46460000E8
:101B2000534552475053202D206261756472617491
:101B300065206F662047505320726563656976653E
:101B400072202834383030206F72203936303020FF
:101B50006F72203139323030290054554E452020E3
:101B6000202D2073657420746865205874616C2082
:101B70006672657175656E63790044415441202039
:101B8000202D206964656E74696669636174696F8C
:101B90006E206F6620726164696F206368697000EF
:101BA000564552202020202D20736F667477617275
:101BB000652076657273696F6E0045584954202020
:101BC000202D20656E64206F6620636F6D6D616EE1
:101BD0006420696E74657270726574657200436822
:101BE0006970205265766973696F6E3A20005061A2
:101BF00072743A2053690000506172742042756912
:101C00006C643A20307800004465736372697074C4
:101C1000696F6E2049643A20307800004375737410
:101C20006F6D65722049643A20307800524F4D2024
:101C300049643A20307800004E4F542056495349A9
:101C4000424C4520534154454C495445530052534E
:101C500053493A20000008000000090000000A0073
:101C600000000B0000000C0000000D0000000E0042
:101C70000000100000001200000014000000170017
:101C800000001A0000001E000000220000002700D3
:101C900000002D00000036000000460000005E003D
:101CA00000007F0000007F0000007F0000000800AF
:101CB0000000090000000A0000000B0000000C00FA
:101CC00000000D0000000E000000100000001200D7
:101CD000000014000000170000001A0000001E00A1
:101CE000000022000000270000002D000000360048
:101CF0000000460000005E0000007F0000007F0042
:101D000000007F00000008000000090000000A0039
:101D100000000B0000000C0000000D0000000E0091
:101D20000000100000001200000014000000170066
:101D300000001A0000001E00000022000000270022
:101D400000002D00000036000000460000005E008C
:101D500000007F0000007F0000007F000000400EB8
:101D60003D6E006A190EAF6E200EAC6E900EAB6E1B
:101D7000190E756E200E726E900E716E0001AB0E14
:101D8000926EB60E936E8F0E946ED20ED36ED26A92
:101D90009B6A796A786AF26AF16AF06A816A010E6E
:101DA000C26E080EC16EAB0EC06E0B0E0F01386F07
:101DB000396B080E3A6FE00E426F416F100E406FA4
:101DC000040E9D6EA06A9F6EA26A030ED56ECD6A48
:101DD000BA6AB16A516B4E6B4A6BC66A6C6AAB9E4B
:101DE000708672987284766A670E756E900E716E48
:101DF00003012A992A97296B1D0E04011F6F4C0EAF
:101E00001E6F94988B885A0E41620AD05A0E426215
:101E100007D05A0E436204D044505A0A000102E02F
:101E2000000E01D0010E3A6E000E03013EB1010E0C
:101E30003A1600012BE0270E156E100E76EC03F01B
:101E40001FEC35F09A0E346E990E336E190E326E09
:101E50007F0E316E00C338F0FFC237F0FEC236F09D
:101E6000FDC235F0EBEC05F00108E5E00201C06BC6
:101E7000970E0201C05D000109E2070E156ED00E3B
:101E800076EC03F00201C02B0001F2E35A0E446E1F
:101E9000436E426E416EB1EC2FF0CEEC1DF00301AB
:101EA0003E510001E8A602D0ADEC41F006EC1CF07A
:101EB00064EF1EF0719E03013D350001D8A0CDD125
:101EC000800E026E400E096E206A40C31FF0066A43
:101ED000056A200E016EB50EC5EC01F0620EC5EC70
:101EE00001F0060EC5EC01F03B0EC5EC01F02C0E26
:101EF000C5EC01F0000EC5EC01F0010EC5EC01F0DF
:101F0000060EC5EC01F0000EC5EC01F0000EC5ECAC
:101F100001F0200EC5EC01F0900EC5EC01F0000EB2
:101F2000C5EC01F0000EC5EC01F0000EC5EC01F0AF
:101F3000000EC5EC01F0000EC5EC01F0000EC5EC82
:101F400001F0000EC5EC01F0800E026E400E096E2D
:101F5000206A40C31FF0066A056A200E016E000E5B
:101F6000C5EC01F0000EC5EC01F0000EC5EC01F06F
:101F7000000EC5EC01F0000EC5EC01F0000EC5EC42
:101F800001F0000EC5EC01F0000EC5EC01F0000EF2
:101F9000C5EC01F0000EC5EC01F0000EC5EC01F03F
:101FA0002C0EC5EC01F0010EC5EC01F0000EC5ECE5
:101FB00001F0000EC5EC01F04F0EC5EC01F0C10EB2
:101FC000C5EC01F0030EC5EC01F0000EC5EC01F00C
:101FD000800E026E400E096E206A40C31FF0066A32
:101FE000056A200E016E860EC5EC01F0020EC5ECEE
:101FF00001F0000EC5EC01F0000EC5EC01F0FE0E84
:10200000C5EC01F0000EC5EC01F0000EC5EC01F0CE
:10201000000EC5EC01F0640EC5EC01F0400EC5ECFD
:1020200001F0010EC5EC01F0000EC5EC01F08F0EC1
:10203000C5EC01F0870EC5EC01F0640E75EC03F001
:10204000800E026E400E096E206A40C31FF0066AC1
:10205000056A200E016EB50EC5EC01F0620EC5ECEE
:1020600001F0060EC5EC01F0160EC5EC01F0080EED
:10207000C5EC01F0000EC5EC01F0000EC5EC01F05E
:10208000030EC5EC01F0030EC5EC01F0000EC5EC2B
:1020900001F0510EC5EC01F0A20EC5EC01F0060EE8
:1020A000C5EC01F0000EC5EC01F0230EC5EC01F00B
:1020B000E70EC5EC01F0640E75EC03F0800E026EC5
:1020C000400E096E206A40C31FF0066A056A200EA2
:1020D000016EB50EC5EC01F0620EC5EC01F0060E06
:1020E000C5EC01F0110EC5EC01F0020EC5EC01F0DB
:1020F000000EC5EC01F0080EC5EC01F0010EC5ECB8
:1021000001F0220EC5EC01F0920EC5EC01F0800E3C
:10211000026E400E096E206A40C31FF0066A056A0F
:10212000200E016E110EF76E060EF66E0900F550C8
:1021300003E0C5EC01F0FAD70D0EC5EC01F00A0E74
:10214000C5EC01F0640E75EC03F0800E026E400EDB
:10215000096E206A40C31FF0066A056A200E016EF0
:10216000110EF76E1E0EF66E0900F55003E0C5EC79
:1021700001F0FAD70D0EC5EC01F00A0EC5EC01F026
:10218000640E75EC03F0800E026E400E096E206A3C
:1021900040C31FF0066A056A200E016E110EF76E2D
:1021A000360EF66E0900F55003E0C5EC01F0FAD7E3
:1021B0000D0EC5EC01F00A0EC5EC01F0640E75ECD5
:1021C00003F0800E026E400E096E206A40C31FF0BD
:1021D000066A056A200E016E110EF76E4E0EF66E3F
:1021E0000900F55003E0C5EC01F0FAD70D0EC5EC7F
:1021F00001F00A0EC5EC01F0640E75EC03F0800EE0
:10220000026E400E096E206A40C31FF0066A056A1E
:10221000200E016E110EF76E660EF66E0900F55077
:1022200003E0C5EC01F0FAD70D0EC5EC01F00A0E83
:10223000C5EC01F0640E75EC03F01AEC47F00301F5
:102240002A510001E8A402D01AEC47F003012A51F8
:102250000001E8A402D01AEC47F003013C51000150
:10226000E8B43CD003013D3500011CE2800E026E53
:10227000400E096E206A40C31FF0066A056A200EF0
:10228000016E110EF76E7E0EF66E0900F55003E03A
:10229000C5EC01F0FAD70D0EC5EC01F00A0EC5EC45
:1022A00001F01BD0800E026E400E096E206A40C302
:1022B0001FF0066A056A200E016E110EF76EB00E51
:1022C000F66E0900F55003E0C5EC01F0FAD70D0EEB
:1022D000C5EC01F00A0EC5EC01F03BD003013D3521
:1022E00000011CE2800E026E400E096E206A40C39F
:1022F0001FF0066A056A200E016E110EF76EC80EF9
:10230000F66E0900F55003E0C5EC01F0FAD70D0EAA
:10231000C5EC01F00A0EC5EC01F01BD0800E026E78
:10232000400E096E206A40C31FF0066A056A200E3F
:10233000016E110EF76EFA0EF66E0900F55003E00D
:10234000C5EC01F0FAD70D0EC5EC01F00A0EC5EC94
:1023500001F003013C310001D8B092EC18F0030108
:102360002D6B140E2C6F640E2E6F0001B4D1040E71
:1023700003013A5D000106E2EA0E156E600E76EC8E
:1023800003F0A9D103013D310001D8A05BD00301C6
:102390003D3500011CE2800E026E400E096E206A7F
:1023A00040C31FF0066A056A200E016E120EF76E1A
:1023B000120EF66E0900F55003E0C5EC01F0FAD7F5
:1023C0000D0EC5EC01F00A0EC5EC01F03BD0800EFD
:1023D000026E400E096E206A40C31FF0066A056A4D
:1023E000200E016EB50EC5EC01F0620EC5EC01F0D9
:1023F000060EC5EC01F0570EC5EC01F0080EC5EC59
:1024000001F0000EC5EC01F0010EC5EC01F0000E6C
:10241000C5EC01F0000EC5EC01F0000EC5EC01F0BA
:10242000500EC5EC01F04F0EC5EC01F0540EC5EC9A
:1024300001F0530EC5EC01F0AC0EC5EC01F0850EB9
:10244000C5EC01F003013E31000120E350EC35F012
:1024500004C334F003C333F002C332F001C331F0DC
:10246000386A376A366A7E0E356EEBEC05F0010885
:1024700007E03A0E04011F6F980E1E6F000105D091
:102480001D0E04011F6F4C0E1E6F0001A20ED36EB5
:10249000D288C2901D0E03012D5D00010FE305E1FE
:1024A0004D0E03012C5D000109E31FC415F004016A
:1024B0001E5176EC03F00001B5EC1DF0130E030184
:1024C0002D5D00010FE305E1890E03012C5D000184
:1024D00009E31FC415F004011E5176EC03F000015E
:1024E000B5EC1DF0090E03012D5D000116E305E1B9
:1024F000C50E03012C5D000110E31FC415F004019B
:102500001E5176EC03F00001B5EC1DF0640E0301E2
:10251000295D000102E20301292B050E03012D5D57
:10252000000113E305E1DD0E03012C5D00010DE365
:102530001FC415F004011E5176EC03F00001B5EC48
:102540001DF003012A9700010BD0040E0301295D41
:10255000000104E303012A87000102D003012A9746
:1025600003012D53000107E1650E03012C5D0001FD
:1025700002E2000E01D0010E3A6E010E03012D5D44
:10258000000108E305E12C0E03012C5D000102E3CC
:10259000000E01D0010E3A16010E03012AB7000EFB
:1025A0003A16000112E01FC415F004011E5176EC2A
:1025B00003F00001B5EC1DF01FC415F004011E511D
:1025C00076EC03F00001B5EC1DF0710E04011E5D08
:1025D000146E020E1F59156E77EC03F0D298D20ECE
:1025E000D36EC28003013D310001D8A05BD003014E
:1025F0003D3500011CE2800E026E400E096E206A1D
:1026000040C31FF0066A056A200E016E120EF76EB7
:10261000200EF66E0900F55003E0C5EC01F0FAD784
:102620000D0EC5EC01F00A0EC5EC01F03BD0800E9A
:10263000026E400E096E206A40C31FF0066A056AEA
:10264000200E016EB50EC5EC01F0620EC5EC01F076
:10265000060EC5EC01F0570EC5EC01F0080EC5ECF6
:1026600001F0000EC5EC01F0010EC5EC01F0000E0A
:10267000C5EC01F0000EC5EC01F0000EC5EC01F058
:10268000200EC5EC01F04E0EC5EC01F0550EC5EC68
:1026900001F0520EC5EC01F07B0EC5EC01F0C30E4B
:1026A000C5EC01F0130E156E880E76EC03F0B5EC58
:1026B0003DF0000E03013CB1010E3A6E000E2AB748
:1026C000010E3A12000107E092EC18F0010E156EAF
:1026D000F40E76EC03F042D8040E03013A5D0001DB
:1026E0003CE3070E156ED00E76EC03F037D81FECE6
:1026F00035F0130E03012D5D000106E307E1890E9D
:1027000003012C5D000102E2000E01D0010E3A6EC1
:1027100000C334F0FFC233F0FEC232F0FDC231F02C
:102720009A0E386E990E376E190E366E7F0E356E14
:1027300023EC06F03A16000110E0070E156ED00EDD
:1027400076EC03F0EBC21AF336C3EBF2A8EC1BF005
:1027500005D81AC3EBF2A8EC1BF009D603013E51D1
:102760000001E8A80AD000EE45F0120EF76E2C0E1C
:10277000F66EBAEC04F0EE6AA7D0800E026E800E00
:10278000096E206A40C31FF00B0E066EB80E056E70
:1027900084EC01F0D8A0D6EF1AF02408F9E184EC1B
:1027A00001F0D8A0D6EF1AF04708F2E184EC01F06E
:1027B000D8A0D6EF1AF05008EBE184EC01F0D8A0D5
:1027C000D6EF1AF04708E4E184EC01F0D8A0D6EF88
:1027D0001AF04708DDE184EC01F0D8A0D6EF1AF03A
:1027E00003011C6F010E256F1CC3F1F00001800E68
:1027F000026E800E096E206A40C31FF0066AC80E82
:10280000056E84EC01F0D8A0A9D703011C6F00EE7F
:10281000F1F025511CC3EBFF252B2A0E1C5DD8A41B
:10282000010E3A6E4F0E255D010ED8B0000E3A161D
:102830000001DCE1800E026E800E096E206A40C34A
:102840001FF0050E396E020E086E08EC00F0030151
:10285000266FF36A00EEF1F02551F3CFEBFF00EEA7
:1028600045F0470EEE6E500EEE6E470EEE6EEE6EBB
:1028700010EEF1F0550EE75204E0E6CFEEFFE82E41
:10288000FAD7EF6A0201C06B03011B6B000100EE77
:1028900045F00201C051EB500C6E2A0E0C5C000199
:1028A0000CE000EE45F00201C051EB500C6E03014C
:1028B0001B1B0201C02B0001E9D703011B51265D40
:1028C0000001D8A4FAEF1AF003013E510001E8A874
:1028D0000AD000EE9BF0120EF76E7A0EF66EBAEC8E
:1028E00004F0EE6AADD003013C510001E8A4DCD055
:1028F000800E026E800E096E206A40C31FF00B0E20
:10290000066EB80E056E84EC01F0D8A0D6EF1AF072
:102910002408F9E184EC01F0D8A0D6EF1AF04708BA
:10292000F2E184EC01F0D8A0D6EF1AF05008EBE108
:1029300084EC01F0D8A0D6EF1AF05608E4E184EC5C
:1029400001F0D8A0D6EF1AF05408DDE184EC01F0D4
:10295000D8A0D6EF1AF003011C6F010E256F1CC31F
:10296000F1F00001800E026E800E096E206A40C3F5
:102970001FF0066AC80E056E84EC01F0D8A0A4D73B
:1029800003011C6F00EEF1F025511CC3EBFF252B5A
:102990002A0E1C5DD8A4010E3A6E4F0E255D010E65
:1029A000D8B0000E3A160001DCE1800E026E800EF7
:1029B000096E206A40C31FF0050E396E020E086EC4
:1029C00008EC00F00301266FF36A00EEF1F02551E8
:1029D000F3CFEBFF00EE9BF0470EEE6E500EEE6E67
:1029E000560EEE6E540EEE6E10EEF1F0550EE752EE
:1029F00004E0E6CFEEFFE82EFAD7EF6A0201C06BE3
:102A000003011B6B000100EE9BF00201C051EB5073
:102A10000C6E2A0E0C5C00010CE000EE9BF0020133
:102A2000C051EB500C6E03011B1B0201C02B0001B7
:102A3000E9D703011B51265D0001D8A42EEF1BF03E
:102A400000EEF1F010EE9BF0550EE75204E0E6CFF9
:102A5000EEFFE82EFAD7EF6A02EE1EF0EF6A02EE02
:102A60002EF0EF6A0201CD6B00016EEC1DF002EE5C
:102A70001EF012EE44F0320EE75204E0E6CFEEFF15
:102A8000E82EFAD7EF6A0201CD6B000174EC1DF05D
:102A900002EE2EF012EE44F0320EE75204E0E6CFE2
:102AA000EEFFE82EFAD7EF6A0301386B00EEF1F083
:102AB00010EE45F0550EE75204E0E6CFEEFFE82EAB
:102AC000FAD7EF6A0201CD6B00016FEC1DF0020135
:102AD0004451BB6F300EBB5D0001D8A45CD03A0EF0
:102AE00003012E5D000105E203012E2B000136D605
:102AF00051D003012D530001D8A44CD0640E030122
:102B00002C5D0001D8B046D002EE3EF0300EEE6EE5
:102B1000EF6A0201CD6B00019AEC1DF000EEF1F0BE
:102B20000201CD51EBCF0CF00CC0DEF1CD2900EE4F
:102B3000F1F0EBCF0CF00CC0DFF13A0E0101E06FC9
:102B4000020E0201CD2500EEF1F0EBCF0CF00CC02F
:102B5000E1F1030ECD2500EEF1F0EBCF0CF00CC04F
:102B6000E2F13A0E0101E36F040E0201CD2500EE01
:102B7000F1F0EBCF0CF00CC0E4F1050ECD2500EE2A
:102B8000F1F0EBCF0CF00CC0E5F10101E66B0001B8
:102B900019D9E4D517D101EEDEF0EF6A01EEEEF0BF
:102BA000EF6A01EEFEF0EF6A02EE3EF0EF6A02011C
:102BB000CD6B00019AEC1DF000EEF1F00201CD5159
:102BC000EBCF0CF00CC0DEF1CD2900EEF1F0EBCF35
:102BD0000CF00CC0DFF13A0E0101E06F020E0201B1
:102BE000CD2500EEF1F0EBCF0CF00CC0E1F1030EBF
:102BF000CD2500EEF1F0EBCF0CF00CC0E2F13A0E77
:102C00000101E36F040E0201CD2500EEF1F0EBCFE0
:102C10000CF00CC0E4F1050ECD2500EEF1F0EBCF89
:102C20000CF00CC0E5F10101E66B0201CD6B000177
:102C300073EC1DF001EEEEF012EE44F0320EE752AE
:102C400004E0E6CFEEFFE82EFAD7EF6A0201CD6B83
:102C5000000172EC1DF002EE44F0EECFF3FFEFCF77
:102C6000F4FFF350530AF4101AE102EE44F02D0E73
:102C7000EE6E11EEEEF00F0EE75204E0E6CFEEFF3F
:102C8000E82EFAD7EF6A01EEEEF012EE44F0320EC3
:102C9000E75204E0E6CFEEFFE82EFAD7EF6A020132
:102CA000CD6B000171EC1DF001EEFEF012EE44F070
:102CB000320EE75204E0E6CFEEFFE82EFAD7EF6AD5
:102CC0000201CD6B000170EC1DF002EE44F0EECF7E
:102CD000F3FFEFCFF4FFF350570AF4101AE102EEBE
:102CE00044F02D0EEE6E11EEFEF00F0EE75204E0F2
:102CF000E6CFEEFFE82EFAD7EF6A01EEFEF012EE15
:102D000044F0320EE75204E0E6CFEEFFE82EFAD7A9
:102D1000EF6A0201CD6B00016EEC1DF002EE3EF099
:102D200012EE44F0320EE75204E0E6CFEEFFE82E5A
:102D3000FAD7EF6A02EE3EF004EC00F003013A6FBE
:102D40000201CD6B00016CEC1DF0040E03013A5D35
:102D5000000114E302EE0EF012EE44F0320EE752E0
:102D600004E0E6CFEEFFE82EFAD7EF6A02EE0EF0AF
:102D700004EC00F003012C6F19C02DF30201FB2BB2
:102D8000000EFC23FCC211F0FBC210F0030E156E06
:102D9000E80E146E43EC04F019C0FCF218C0FBF20C
:102DA00003013C510001E8BC0DD002EE3EF0020EE2
:102DB000016E030E086EFCC219F0FBC218F0A9ECFC
:102DC00000F0EF6A03012E6B000E3CB7010E3A6E65
:102DD000000E3CB3010E3A120001D8A41FEC35F0EE
:102DE000000E03013DB3010E3A6E000E3CB9010E18
:102DF0003A12000104E0F2EC1BF008EC34F0B5EC00
:102E00003DF001EE47F0240EEE6EEE6EEE6EEE6ECD
:102E100012EE77F0110EE75204E0E6CFEEFFE82E57
:102E2000FAD72C0EEE6E12EE3EF0050EE75204E0DD
:102E3000E6CFEEFFE82EFAD72C0EEE6E11EEDEF0A6
:102E40000F0EE75204E0E6CFEEFFE82EFAD72C0E85
:102E5000EE6E11EEEEF00F0EE75204E0E6CFEEFF5D
:102E6000E82EFAD72C0EEE6E11EEFEF00F0EE752A2
:102E700004E0E6CFEEFFE82EFAD72C0EEE6E12EE4F
:102E80000EF00F0EE75204E0E6CFEEFFE82EFAD781
:102E9000EF6A03012A510001E8B6F5D003013E5163
:102EA0000001E8A617D010EC42F001EE47F0EE501A
:102EB000FEE1ED522C0EEE6E020E016ED9C326F02D
:102EC000D8C325F0D7C324F0D6C323F0010EE3EC1A
:102ED00000F0EF6A03013C510001E8A41CD001EEB0
:102EE00047F0EE50FEE1ED522C0EEE6E12EE1EF0AB
:102EF0000F0EE75204E0E6CFEEFFE82EFAD72C0ED5
:102F0000EE6E12EE2EF00F0EE75204E0E6CFEEFF6B
:102F1000E82EFAD7EF6A03013C510001E8AA17D066
:102F20008DEC34F001EE47F0EE50FEE1ED522C0E48
:102F3000EE6E020E016E0AC326F009C325F008C327
:102F400024F007C323F0010EE3EC00F0EF6A030165
:102F50003D510001E8A215D001EE47F0EE50FEE130
:102F6000ED522C0EEE6E020E016E0EC326F00DC356
:102F700025F00CC324F00BC323F0010EE3EC00F0AA
:102F8000EF6A03013C35000117E3D6EC34F001EEA3
:102F900047F0EE50FEE1ED522C0EEE6E020E016E89
:102FA00012C326F011C325F010C324F00FC323F081
:102FB000030EE3EC00F0EF6A03013C510001E8A8C6
:102FC00014D001EE47F0EE50FEE1ED522C0EEE6E05
:102FD000020E016E16C326F015C325F014C324F0AB
:102FE00013C323F0E3EC00F0EF6A03013C5100014E
:102FF000E8A614D001EE47F0EE50FEE1ED522C0EA3
:10300000EE6E020E016E00C326F0FFC225F0FEC276
:1030100024F0FDC223F0E3EC00F0EF6A03013E313F
:10302000000131E381EC35F003013E510001E8A2DB
:1030300014D001EE47F0EE50FEE1ED522C0EEE6E94
:10304000020E016E04C326F003C325F002C324F070
:1030500001C323F0E3EC00F0EF6A03013E510001ED
:10306000E8A411D001EE47F0EE50FEE1ED522C0E37
:10307000EE6E020E016E086A06C319F005C318F061
:10308000A4EC00F0EF6A03013D510001E8A413D065
:1030900043EC3AF001EE47F0EE50FEE1ED522C0E1B
:1030A000EE6E12EE44F0320EE75204E0E6CFEEFF91
:1030B000E82EFAD7EF6A03011B6B01EE47F0E86ACE
:1030C000EE5202E0E83EFCD70B6E040E0201CD6F1B
:1030D0000201CD510B5C00010FE301EE47F002014C
:1030E000CD51E926000EEA22EF500C6E03011B1BA6
:1030F0000201CD2B0001ECE301EE47F0EE50FEE1C2
:10310000ED522A0EEE6E020E016E086E03011B5187
:103110008AEC00F00D0EEE6E0A0EEE6EEF6A000104
:103120000CEF1DF003012E6B2A93300E0201BB6FD2
:1031300003013D510001E8A8CBD003013E5100013D
:10314000E8A80AD000EEF1F0120EF76E2C0EF66E23
:10315000BAEC04F0EE6AA7D0800E026E800E096E03
:10316000206A40C31FF00B0E066EB80E056E84EC8D
:1031700001F0D8A0ADD02408FAE184EC01F0D8A089
:10318000A7D04708F4E184EC01F0D8A0A1D0500802
:10319000EEE184EC01F0D8A09BD04708E8E184EC94
:1031A00001F0D8A095D04708E2E184EC01F0D8A066
:1031B0008FD003011C6F010E256F1CC3F1F00001BD
:1031C000800E026E800E096E206A40C31FF0066AF0
:1031D000C80E056E84EC01F0D8A0AEEF13F0030129
:1031E0001C6F00EEF1F025511CC3EBFF252B2A0EBE
:1031F0001C5DD8A4010E3A6E4F0E255D010ED8B0AD
:10320000000E3A160001DBE1800E026E800E096EA0
:10321000206A40C31FF0050E396E020E086E08ECDE
:1032200000F00301266FF36A00EEF1F02551F3CFB1
:10323000EBFF00EE45F0470EEE6E500EEE6E470EC1
:10324000EE6EEE6E10EEF1F0550EE75204E0E6CFB2
:10325000EEFFE82EFAD7EF6A0201C06B03011B6B89
:10326000000100EE45F00201C051EB500C6E2A0E39
:103270000C5C00010CE000EE45F00201C051EB5087
:103280000C6E03011B1B0201C02B0001E9D70301D7
:103290001B51265D000107E003012E2B050E2E5D5C
:1032A0000001D8A04AD70201CD6B00016FEC1DF0E0
:1032B00002014451BB6F300EBB5D000109E1030107
:1032C0002A510001E8B204D003012A83000135D756
:1032D000B5EC3DF093968A9614DAC5EC1BF002012A
:1032E000C06B0001AA6A100E0201C025A96ED8B0F9
:1032F000AA2AF2EC02F0EC6FC02B200EEC5D00016C
:103300000BE103012851050DF3CF14F0F4CF15F0B4
:1033100077EC03F00001E5D70201EC29010ED8A4F7
:10332000000E3A6E100EC05D000102E2000E01D0E8
:10333000010E3A1202E1DDD8D4D703012A5100016F
:10334000E8B682D003013D510001E8AC30D0030E55
:10335000156EE80E76EC03F002EE44F0550EEE6EBC
:10336000020E016E00C326F0FFC225F0FEC224F05B
:10337000FDC223F0E3EC00F0560EEE6EEF6A0201A0
:10338000C06B000102EE44F00201C051EB500C6E24
:103390000C5200010CE002EE44F00201C051EB506F
:1033A000EC6F0001A6D80201C02B0001EAD703018F
:1033B0003C510001E8A248D002EE2EF0020E016E50
:1033C0000AC326F009C325F008C324F007C323F07D
:1033D000010EE3EC00F0EF6A02012E510C6E2D0E8F
:1033E0000C5C000103E14E0E02012E6F0001030E82
:1033F000156EE80E76EC03F002EE44F0540EEE6E1D
:1034000012EE2EF00F0EE75204E0E6CFEEFFE82EAC
:10341000FAD7430EEE6EEF6A0201C06B000102EEB6
:1034200044F00201C051EB500C6E0C5200010CE054
:1034300002EE44F00201C051EB50EC6F000159D88C
:103440000201C02B0001EAD7000E03013DB9010EB5
:103450003A6E000E2AB7010E3A120001D8B443D0DA
:10346000300E0201BB5D00013EE00201CD6B0001A8
:103470006CEC1DF002EE44F004EC00F003012C6F44
:1034800019C02DF3000143EC3AF002EE44F0EE5087
:10349000FEE1ED52200EEE6E020E016E086A2DC3A3
:1034A00019F02CC318F0A9EC00F0EF6A030E156EAA
:1034B000E80E76EC03F00201C06B000102EE44F06E
:1034C0000201C051EB500C6E0C5200010CE002EEF8
:1034D00044F00201C051EB50EC6F00010AD8020128
:1034E000C02B0001EAD75BD9030E156EE80E76EF0C
:1034F00003F0410E0201EC5D000112E2246A900E1D
:103500000201EC25236ED8B0242A2E0E235CEE6F28
:10351000AA6AEEC2A9FFF2EC02F0EB6F000110D034
:10352000246AA00E0201EC25236ED8B0242A410E95
:10353000235CEE6FAA6AEEC2A9FFF2EC02F0EB6F19
:103540000201EB510001E8BE26D0020E0201EB5D44
:10355000000121E393968A860201EB3100010BE31F
:1035600003012851030DF3CF14F0F4CF15F077ECDD
:1035700003F0000104D00301285175EC03F00001B1
:1035800093968A960301285175EC03F0D8900201B6
:10359000EB330001D5D703012851020DF3CF14F00E
:1035A000F4CF15F077EC03F000011200949494949A
:1035B0008B94640E75EC03F094840301382B060E93
:1035C000385D000115E301EE47F00D0EEE6E0A0EB8
:1035D000EE6E120EF76EA00EF66EBAEC04F00D0E43
:1035E000EE6E0A0EEE6EEF6A0301386B000114D224
:1035F000AEEF13F00301382B060E385D00012CE30B
:1036000001EE47F00D0EEE6E0A0EEE6E120EF76E24
:10361000C00EF66EBAEC04F0240EEE6E470EEE6E9F
:10362000500EEE6E470EEE6EEE6E10EEF1F0550E91
:10363000E75204E0E6CFEEFFE82EFAD7200EEE6E5A
:10364000EE6E0D0EEE6E0A0EEE6EEF6A0301386B33
:103650000001EFEC39F0E0D1AEEF13F00301382BAD
:10366000060E385D00012DE301EE47F00D0EEE6E03
:103670000A0EEE6E120EF76EC00EF66EBAEC04F085
:10368000240EEE6E470EEE6E500EEE6E560EEE6E81
:10369000540EEE6E10EEF1F0550EE75204E0E6CF58
:1036A000EEFFE82EFAD7200EEE6EEE6E0D0EEE6EE9
:1036B0000A0EEE6EEF6A0301386B0001EFEC39F091
:1036C000ABD1AEEF13F0050E0201896F110E8A6FB8
:1036D000200E8B6F010E8C6F8D6B8A0E8E6F00012A
:1036E00040EF3FF0050E0201896F110E8A6F200E28
:1036F0008B6F010E8C6F8D6B880E8E6F000140EF0B
:103700003FF0050E0201896F110E8A6F200E8B6F3C
:10371000010E8C6F8D6B890E8E6F000140EF3FF0B4
:10372000080E0201896F130E8A6F040E8B6F150E3F
:103730008C6F210E8D6F200E8E6F080E8F6F0B0E0B
:10374000906F916B140E75EC03F0000142EF3FF0A7
:10375000050E0201896F110E8A6F220E8B6F010E0A
:103760008C6F8D6FEBC28EF2000140EF3FF0050EC3
:103770000201896F110E8A6F8B6B010E8C6F8D6B3E
:10378000ECC28EF2000140EF3FF0020E0201896FA1
:10379000340E8A6F070E8B6F000140EF3FF0020E70
:1037A0000201896F340E8A6F010E8B6F000140EFAA
:1037B0003FF0020E0201896F340E8A6F050E8B6F87
:1037C000000140EF3FF0060E0201896F310E8A6F53
:1037D000010E8B6F300E8C6F8D6B8E6B8F6B0001BB
:1037E00040EF3FF0020E0201896F340E8A6F030E24
:1037F0008B6F000140EF3FF0020E0201896F340E23
:103800008A6F080E8B6F000140EF3FF0080E020137
:10381000896F320E8A6F8B6B8C6B8D6B8E6B8F6B9F
:10382000906B916B000140EF3FF0020E0201896F37
:10383000340E8A6F060E8B6F000140EF3FF0020ED0
:103840000201896F340E8A6F020E8B6F000140EF08
:103850003FF0D9C232F0D8C231F03CEC08F0C8C217
:1038600038F0C7C237F0C6C236F0C5C235F09BEC9F
:1038700007F0E9EC07F00201EF6F32C0F0F200014F
:10388000EFC2E7F2F0C2E8F2060E0201896F110EF4
:103890008A6F200E8B6F020E8C6F0D0E8D6FE8C23B
:1038A0008EF2E7C28FF2000140EF3FF0C8C226F06F
:1038B000C7C225F0C6C224F0C5C223F030C332F01F
:1038C0002FC331F044EC08F034C02AF033C029F0A3
:1038D00032C028F031C027F0346A336A326A7F0E72
:1038E000316E2AC038F029C037F028C036F027C022
:1038F00035F0A7EC06F034C02AF033C029F032C00E
:1039000028F031C027F02752D8B43D84D8A4270628
:1039100026C038F025C037F024C036F023C035F07B
:103920002AC034F029C033F028C032F027C031F06B
:103930009BEC07F0E9EC07F00201F56F32C0F6F2FC
:10394000F6C2EAF2F5C2E9F2070E896F110E8A6F2C
:10395000200E8B6F030E8C6F0A0E8D6F8E6BEAC27A
:103960008FF2E9C290F2000140EF3FF0050E020134
:10397000896F110E8A6F200E8B6F010E8C6F1A0EDD
:103980008D6F8E6B000140EC3FF0136A080E126ED3
:10399000116A106A1B6A1A6A196ACEC218F05AECC8
:1039A00004F013C0DFF212C0DEF211C0DDF210C06D
:1039B000DCF2DFC213F0DEC212F0DDC211F0DCC2B5
:1039C00010F01B681A681968186AB8EC03F013C085
:1039D000DFF212C0DEF211C0DDF210C0DCF2DEC296
:1039E00041F3DDC242F3DCC243F3030E030141178E
:1039F000060E0201896F110E8A6F200E8B6F030E67
:103A00008C6F1B0E8D6F41C38EF242C38FF243C386
:103A100090F2000140EF3FF093968A8654DEB5DEC7
:103A2000640E75EC03F00201C06B000101EE47F07B
:103A30000201C051E926000EEA22EF500C6E000E82
:103A40000C52D8A4010E3A6E960EC05D010ED8B08D
:103A5000000E3A16000110E001EE47F00201C051DD
:103A6000E926000EEA22EF500301276F000108D873
:103A70000201C02B0001D9D7640E75EC03F08FD67C
:103A800093968A96F8C211F00201F75183EC03F085
:103A9000010E03011C6F03011C51335D000112E391
:103AA000030127B1818627A18196F8C211F0020196
:103AB000F75183EC03F0D8900301273303011C2B4B
:103AC0000001E9E393968A86FAC211F00201F951E6
:103AD00083EC03F0000112002DD82CD82BD82AD863
:103AE00029D828D827D826D825D80201C06B0001AC
:103AF00000EEF1F00201CD51EB500C6E2C0E0C5C7F
:103B000000010FE000EEF1F00201CD51EBCF0CF01F
:103B100002EE44F0C0510CC0EBFFC02BCD2B0001D6
:103B2000E6D7F36A02EE44F00201C051F3CFEBFF97
:103B30000001120000EEF1F00201CD51EB500C6ECD
:103B40002C0E0C5CD8A4010E3A6E500ECD5D010E09
:103B5000D8B0000E3A16000104E00201CD2B00019E
:103B6000E9D70201CD2B0001120093968A8681ECE1
:103B70001BF00BDE1D0E116E4C0E83EC03F09396C2
:103B80008A961D0E116E4C0E83EC03F093968A8676
:103B90001D0E116E4C0E83EC03F001D6D7C2E6F277
:103BA000D6C2E5F2D5C2E4F2D4C2E3F2640E75ECFB
:103BB00003F094988B88020E156E580E76EC03F085
:103BC00094988B98949A8B9A820E026E400E096E8E
:103BD000810E036E010E046E0A6E106E4AEC03F045
:103BE000949A8B8AC80E75EC03F0070E0201896F58
:103BF000020E8A6F010E8B6F8C6BE6C28DF2E5C2EE
:103C00008EF2E4C28FF2E3C290F203013D51000153
:103C1000E8A603D0010E02018C6F000142EC3FF0D8
:103C2000140E75EC03F0040E0201896F200E8A6FEA
:103C30008B6B8C6B8D6B000142EC3FF0140E75ECBE
:103C400003F090EC1BF0B9EC3FF003DE2FDE080E22
:103C50000201CF2503011C6F050E0201896F110EB1
:103C60008A6F200E8B6F010E8C6F510E8D6F1CC3EF
:103C70008EF2000140EC3FF0050E0201896F110E3B
:103C80008A6F220E8B6F010E8C6F8D6B080E8E6FFC
:103C9000000140EC3FF0A8EC1BF003013D51000196
:103CA000E8A602D00201EC6B0001B7EC1BF0050E98
:103CB0000201896F110E8A6F8B6B010E8C6F8D6FF5
:103CC0008E6F000140EF3FF0AE6A0D0E64EC02F023
:103CD000120EF76ED60EF66E5CEC02F0016A086A00
:103CE000196A040E186EA9EC00F02E0E64EC02F0B6
:103CF000010E086E2D0EA7EC00F0120EF76EEA0E04
:103D0000F66E5CEC02F00D0E64EC02F0130E096E20
:103D1000880E026E37EC02F0D8A05AEF0FF00301C4
:103D20003B6F120EF76EF60EF66E5CEC02F00D0EA7
:103D300064EC02F0630E64EC02F06D0E64EC02F0D1
:103D4000640E64EC02F03E0E64EC02F0000103D855
:103D50006ED8D1D8FBD7130E096E880E026E37ECE1
:103D600002F0F9E303013B6F3B5164EC02F00D0EEE
:103D70003B5D010ED8A4000E3A6E0A0E3B5D010EAB
:103D8000D8A4000E3A120001D8A41200010E0301BB
:103D9000256F3BC3F1F00001130E096E880E026E11
:103DA00037EC02F03AE303013B6F3B5164EC02F065
:103DB000080E3B5D000108E103012553000102E00C
:103DC000030125070001E7D70D0E03013B5D010E3E
:103DD000D8A4000E3A6E0A0E3B5D010ED8A4000E68
:103DE0003A122529010ED8A4000E3A1200010BE068
:103DF0000D0EF36E00EEF1F003012551F3CFEBFF52
:103E00000001120006D000EEF1F0030125513BC382
:103E1000EBFF0301252B0001BED70D0EF36E00EE64
:103E2000F1F003012551F3CFEBFF00011200020175
:103E3000CD6B000100EEF1F00201CD51EB500C6EA4
:103E4000200E0C5CD8A4010E3A6E00EEF1F0CD51BC
:103E5000EB500C6E0D0E0C5CD8A4010E3A16FD0E44
:103E6000CD5D010ED8B0000E3A1600013AE000EE2A
:103E7000F1F00201CD51EB500C6E610E0C5C000EA6
:103E8000D8B0010E3A6E00EEF1F0CD51EB500C6E51
:103E90007B0E0C5C000102E3000E01D0010E3A160D
:103EA0000EE000EEF1F00201CD51EB500E6EDF0E90
:103EB0000E140C6E00EEF1F0CD510CC0EBFF0001C2
:103EC00000EEF1F00201CD51EBCF0CF001EE47F026
:103ED000CD51E926000EEA220CC0EFFFCD2B0001E8
:103EE000A8D701EE47F00201CD51E926000EEA22E3
:103EF000EF6A00011200F1510C6E0A0E0C5C010E0B
:103F0000D8A4000E3A6EF1510C6E0D0E0C5C010E31
:103F1000D8A4000E3A12D8A41200130EF76E0A0E9F
:103F2000F66E01EE47F0C2EC04F002E12FD213D29C
:103F3000130EF76E100EF66E01EE47F0C2EC04F0B1
:103F400009E0130EF76E140EF66E01EE47F0C2ECA8
:103F500004F003E135EF2BF0FED1130EF76E1C0ECB
:103F6000F66E01EE47F0C2EC04F009E0130EF76EB6
:103F7000200EF66E01EE47F0C2EC04F003E1CBEF49
:103F800023F0E9D1130EF76E260EF66E01EE47F020
:103F9000C2EC04F003E19BEF23F0DDD1130EF76ECA
:103FA0002E0EF66E01EE47F0C2EC04F003E1B3EF23
:103FB00023F0D1D1130EF76E340EF66E01EE47F0FA
:103FC000C2EC04F003E167EF2BF0C5D1130EF76EDE
:103FD0003A0EF66E01EE47F0C2EC04F009E0130E63
:103FE000F76E3E0EF66E01EE47F0C2EC04F003E110
:103FF0000EEF28F0B0D1130EF76E480EF66E01EEFC
:1040000047F0C2EC04F009E0130EF76E4C0EF66EAA
:1040100001EE47F0C2EC04F003E145EF2AF09BD13A
:10402000130EF76E560EF66E01EE47F0C2EC04F07A
:1040300009E0130EF76E5C0EF66E01EE47F0C2EC6F
:1040400004F003E179EF2AF086D1130EF76E620EC9
:10405000F66E01EE47F0C2EC04F003E1B7EF2AF090
:104060007AD1130EF76E680EF66E01EE47F0C2ECD1
:1040700004F003E1C7EF2AF06ED1130EF76E6E0E57
:10408000F66E01EE47F0C2EC04F009E0130EF76E95
:10409000740EF66E01EE47F0C2EC04F003E190EF0F
:1040A0002BF059D1130EF76E7A0EF66E01EE47F033
:1040B000C2EC04F009E0130EF76E800EF66E01EE0E
:1040C00047F0C2EC04F003E103EF2BF044D1130EF0
:1040D000F76E860EF66E01EE47F0C2EC04F003E1D7
:1040E0003BEF23F038D1130EF76E8C0EF66E01EE17
:1040F00047F0C2EC04F003E153EF23F02CD1130E90
:10410000F76E920EF66E01EE47F0C2EC04F003E19A
:104110006BEF23F020D1130EF76E980EF66E01EEC2
:1041200047F0C2EC04F003E183EF23F014D1130E47
:10413000F76EA00EF66E01EE47F0C2EC04F002E15D
:1041400088D109D1130EF76EA60EF66E01EE47F078
:10415000C2EC04F002E195D1FED0130EF76EAC0E66
:10416000F66E01EE47F0C2EC04F002E1A2D1F3D00A
:10417000130EF76EB40EF66E01EE47F0C2EC04F0CB
:1041800002E1AFD1E8D0130EF76EBC0EF66E01EE71
:1041900047F0C2EC04F002E126D2DDD0130EF76E38
:1041A000C20EF66E01EE47F0C2EC04F002E1EBD174
:1041B000D2D0130EF76EC80EF66E01EE47F0C2ECC9
:1041C00004F002E1F8D1C7D0130EF76ECE0EF66EF2
:1041D00001EE47F0C2EC04F003E1FBEF23F0BBD0AB
:1041E000130EF76ED40EF66E01EE47F0C2EC04F03B
:1041F00003E1A3EF24F0AFD0130EF76EDA0EF66EE4
:1042000001EE47F0C2EC04F003E1F4EF28F0A3D094
:10421000130EF76EDE0EF66E01EE47F0C2EC04F000
:1042200003E1E3EF23F097D0130EF76EE40EF66E82
:1042300001EE47F0C2EC04F003E1BDEF29F08BD0B2
:10424000130EF76EEC0EF66E01EE47F0C2EC04F0C2
:1042500003E189EF2DF07FD0130EF76EF20EF66EAC
:1042600001EE47F0C2EC04F003E15BEF2CF073D0F9
:10427000130EF76EF80EF66E01EE47F0C2EC04F086
:1042800002E19ED068D0130EF76EFE0EF66E01EEC0
:1042900047F0C2EC04F003E115EF24F05CD0140EFB
:1042A000F76E040EF66E01EE47F0C2EC04F003E187
:1042B00043EF24F050D0140EF76E0A0EF66E01EEA6
:1042C00047F0C2EC04F002E195D045D0140EF76E31
:1042D000120EF66E01EE47F0C2EC04F003E119EFA6
:1042E0002CF039D0140EF76E1C0EF66E01EE47F06E
:1042F000C2EC04F003E191EF2CF02DD0140EF76E18
:10430000220EF66E01EE47F0C2EC04F002E183D11A
:1043100022D0140EF76E280EF66E01EE47F0C2ECB6
:1043200004F002E190D117D0140EF76E2E0EF66E47
:1043300001EE47F0C2EC04F003E12CEF2CF00BD0BF
:10434000140EF76E320EF66E01EE47F0C2EC04F07A
:10435000D8B449EF2CF0140EF76E380EF66E5CEC04
:1043600002F00D0E64EC02F0630E64EC02F06D0ED0
:1043700064EC02F0640E64EC02F03E0E64EC02F0B9
:10438000640E75EC03F074CF1CF31200DDEC2EF01C
:104390001BEC2DF003012A310001D8B023EF2FF0E0
:1043A00003012A31E832D8B03C81D8A03C91AA6AF6
:1043B000800EA96E3C51F9EC02F0000142EF2FF0A3
:1043C000DDEC2EF01BEC2DF003012A310001D8B0FA
:1043D00023EF2FF003012A31E832D8B03D81D8A075
:1043E0003D91AA6A810EA96E3D51F9EC02F00001DF
:1043F00042EF2FF059EC2FF003011D51300A1E112E
:10440000000105E1BC0E0301406F000118D003015B
:104410001D51600A1E11000105E1500E0301406F9D
:1044200000010DD003011D51C00A1E11000105E15C
:104430001E0E0301406F000102D023EF2FF0AA6A85
:10444000890EA96E03014051F9EC02F0000142EF20
:104450002FF01BEC2DF003012A310001D8B023EF1F
:104460002FF003012A31E832D8B03E87D8A03E971A
:10447000AA6A820EA96E3E51F9EC02F0000142EFE9
:104480002FF01BEC2DF003012A310001D8B023EFEF
:104490002FF003012A31E832D8B03D8DD8A03D9DE0
:1044A000AA6A810EA96E3D51F9EC02F0000142EFBB
:1044B0002FF01BEC2DF003012A310001D8B023EFBF
:1044C0002FF003012A31E832D8B03C83D8A03C93C6
:1044D000AA6A800EA96E3C51F9EC02F0000142EF8D
:1044E0002FF01BEC2DF003012A310001D8B023EF8F
:1044F0002FF003012A31E832D8B03C85D8A03C9592
:10450000AA6A800EA96E3C51F9EC02F03C51000100
:10451000E8B41CD0800E026E400E096E206A40C3C3
:104520001FF0066A056A200E016E110EF76E7E0EF0
:10453000F66E0900F55003E0C5EC01F0FAD70D0E58
:10454000C5EC01F00A0EC5EC01F01BD0800E026E26
:10455000400E096E206A40C31FF0066A056A200EED
:10456000016E110EF76EC80EF66E0900F55003E0ED
:10457000C5EC01F0FAD70D0EC5EC01F00A0EC5EC42
:1045800001F042EF2FF01BEC2DF003012A31000166
:10459000D8B023EF2FF003012A31E832D8B03C899C
:1045A000D8A03C99AA6A800EA96E3C51F9EC02F0A1
:1045B000000142EF2FF01BEC2DF003012A31000126
:1045C000D8B023EF2FF003012A31E832D8B03E856E
:1045D000D8A03E95AA6A800EA96E3C51F9EC02F073
:1045E000000142EF2FF01BEC2DF003012A310001F6
:1045F000D8B023EF2FF003012A31E832D8B03C873E
:10460000D8A03C97AA6A800EA96E3C51F9EC02F042
:10461000000142EF2FF01BEC2DF003012A310001C5
:10462000D8B023EF2FF003012A31E832D8B03E8909
:10463000D8A03E99AA6A820EA96E3E51F9EC02F00A
:10464000000142EF2FF01BEC2DF003012A31000195
:10465000D8B023EF2FF003012A31E832D8B03D8FD4
:10466000D8A03D9FAA6A820EA96E3E51F9EC02F0D5
:10467000000142EF2FF01BEC2DF003012A31000165
:10468000D8B023EF2FF003012A31E832D8B03E81B1
:10469000D8A03E91AA6A820EA96E3E51F9EC02F0B2
:1046A000000142EF2FF01BEC2DF003012A31000135
:1046B000D8B023EF2FF003012A31E832D8B03E837F
:1046C000D8A03E93AA6A810EA96E3D51F9EC02F082
:1046D000000142EF2FF01BEC2DF003012A31000105
:1046E000D8B023EF2FF003012A31E832D8B03C8B49
:1046F000D8A03C9BAA6A800EA96E3C51F9EC02F04E
:10470000000142EF2FF01BEC2DF003012A310001D4
:10471000D8B023EF2FF003012A31E832D8B03D831F
:10472000D8A03D93AA6A810EA96E3D51F9EC02F022
:10473000000142EF2FF01BEC2DF003012A310001A4
:10474000D8B023EF2FF003012A31E832D8B03D85ED
:10475000D8A03D95AA6A810EA96E3D51F9EC02F0F0
:10476000000142EF2FF01BEC2DF003012A31000174
:10477000D8B023EF2FF003012A31E832D8B03D8BB7
:10478000D8A03D9BAA6A810EA96E3D51F9EC02F0BA
:10479000000142EF2FF01BEC2DF003012A31000144
:1047A000D8B023EF2FF003012A31E832D8B03D8989
:1047B000D8A03D99AA6A810EA96E3D51F9EC02F08C
:1047C000000142EF2FF01BEC2DF003012A31000114
:1047D000D8B023EF2FF003012A31E832D8B03D875B
:1047E000D8A03D97AA6A810EA96E3D51F9EC02F05E
:1047F000000142EF2FF01BEC2DF003012A310001E4
:10480000D8B023EF2FF0E86A03012AB3010E010AA2
:10481000D8B43C9DD8A43C8DAA6A800EA96E3C51A8
:10482000F9EC02F0000142EF2FF0DDEC2EF0F15137
:104830000C6E300E0C5CD8B4DEEF35F0F1510C6E1E
:10484000310E0C5CD8B498EF36F0F1510C6E320E8C
:104850000C5CD8B482EF37F0F1510C6E330E0C5C67
:10486000D8B438EF38F0F1510C6E340E0C5CD8B47B
:10487000DDEF38F0F1510C6E350E0C5CD8B436EF2C
:1048800039F023EF2FF0140EF76E4E0EF66E5CEC3F
:1048900002F00D0E64EC02F093968A8672EC1BF027
:1048A000E3EC1BF00B0E096EB80E026E37EC02F053
:1048B000F9E303011C6F550E1C5D010ED8A4000E18
:1048C0003A6E750E1C5D010ED8A4000E3A1200015E
:1048D00006E00201EC53000102E00201EC07440E85
:1048E00003011C5D010ED8A4000E3A6E640E1C5D1F
:1048F000010ED8A4000E3A12000107E07F0E02015B
:10490000EC5D000102E20201EC2B450E03011C5D8F
:10491000010ED8A4000E3A6E650E1C5D010ED8A4DF
:10492000000E3A1200010CE0CFEC1BF0AA6A8A0ECE
:10493000A96E0201EC51F9EC02F0000142EF2FF0F8
:10494000B7EC1BF0AFD70D0E64EC02F0140EF76E4F
:10495000720EF66E5CEC02F003013D35000107E3D8
:104960004F0E64EC02F04E0E64EC02F008D04F0ED5
:1049700064EC02F0460E64EC02F064EC02F00D0E02
:1049800064EC02F0140EF76E7A0EF66E5CEC02F038
:1049900003013E31000107E34F0E64EC02F04E0EBE
:1049A00064EC02F008D04F0E64EC02F0460E64ECAA
:1049B00002F064EC02F00D0E64EC02F0140EF76EDF
:1049C000860EF66E5CEC02F003013C510001E8AA91
:1049D00007D04F0E64EC02F04E0E64EC02F008D0EB
:1049E0004F0E64EC02F0460E64EC02F064EC02F050
:1049F0000D0E64EC02F0140EF76E940EF66E5CEC85
:104A000002F003013D510001E8A207D04F0E64EC13
:104A100002F04E0E64EC02F008D04F0E64EC02F08F
:104A2000460E64EC02F064EC02F00D0E64EC02F051
:104A3000140EF76EAA0EF66E5CEC02F003013C5108
:104A40000001E8A407D04F0E64EC02F04E0E64ECB7
:104A500002F008D04F0E64EC02F0460E64EC02F057
:104A600064EC02F00D0E64EC02F0140EF76EBA0E58
:104A7000F66E5CEC02F003013C510001E8A607D0A1
:104A80004F0E64EC02F04E0E64EC02F008D04F0EB4
:104A900064EC02F0460E64EC02F064EC02F00D0EE1
:104AA00064EC02F0140EF76EC60EF66E5CEC02F0CB
:104AB00003013C510001E8A807D04F0E64EC02F05E
:104AC0004E0E64EC02F008D04F0E64EC02F0460E7D
:104AD00064EC02F064EC02F00D0E64EC02F0140ED3
:104AE000F76ED60EF66E5CEC02F003013E5100014B
:104AF000E8A207D04F0E64EC02F04E0E64EC02F018
:104B000008D04F0E64EC02F0460E64EC02F064EC48
:104B100002F00D0E64EC02F0140EF76EE40EF66E69
:104B20005CEC02F003013E510001E8A407D04F0EF7
:104B300064EC02F04E0E64EC02F008D04F0E64EC10
:104B400002F0460E64EC02F064EC02F00D0E64EC30
:104B500002F0140EF76EF20EF66E5CEC02F003013A
:104B60003C510001E8BC07D04F0E64EC02F04E0E41
:104B700064EC02F008D04F0E64EC02F0460E64ECD8
:104B800002F064EC02F00D0E64EC02F0430E64ECF3
:104B900002F0570E64EC02F0490E64EC02F0440E91
:104BA00064EC02F0200E64EC02F003013C310001E1
:104BB00009E24F0E64EC02F0460E64EC02F064EC85
:104BC00002F006D04F0E64EC02F04E0E64EC02F0E0
:104BD0000D0E64EC02F0140EF76EFC0EF66E5CEC3B
:104BE00002F003013D510001E8AC07D04F0E64EC28
:104BF00002F04E0E64EC02F008D04F0E64EC02F0AE
:104C0000460E64EC02F064EC02F00D0E64EC02F06F
:104C1000150EF76E040EF66E5CEC02F003013C51CB
:104C20000001E8A207D04F0E64EC02F04E0E64ECD7
:104C300002F008D04F0E64EC02F0460E64EC02F075
:104C400064EC02F00D0E64EC02F0150EF76E0C0E23
:104C5000F66E5CEC02F003013D510001E8A407D0C0
:104C60004F0E64EC02F04E0E64EC02F008D04F0ED2
:104C700064EC02F0460E64EC02F064EC02F00D0EFF
:104C800064EC02F0150EF76E160EF66E5CEC02F098
:104C900003013D510001E8AA07D04F0E64EC02F079
:104CA0004E0E64EC02F008D04F0E64EC02F0460E9B
:104CB00064EC02F064EC02F00D0E64EC02F0150EF0
:104CC000F76E1E0EF66E5CEC02F003013D51000122
:104CD000E8A807D04F0E64EC02F04E0E64EC02F030
:104CE00008D04F0E64EC02F0460E64EC02F064EC67
:104CF00002F00D0E64EC02F0150EF76E260EF66E45
:104D00005CEC02F003013D31000107E34F0E64EC5F
:104D100002F04E0E64EC02F008D04F0E64EC02F08C
:104D2000460E64EC02F064EC02F00D0E64EC02F04E
:104D3000150EF76E2E0EF66E5CEC02F003011E6B84
:104D40001D6B1EC320F31DC31FF3040E0301205D62
:104D5000000115E220C3AAFF1FC3A9FFF2EC02F075
:104D600003011C6F1C2900010AE003011C5164ECC3
:104D700002F003011F2B000E20230001E6E30D0EBD
:104D800064EC02F0150EF76E360EF66E5CEC02F077
:104D900003011E6B100E1D6F1EC320F31DC31FF3F6
:104DA000040E0301205D000115E220C3AAFF1FC30A
:104DB000A9FFF2EC02F003011C6F1C2900010AE0BC
:104DC00003011C5164EC02F003011F2B000E202391
:104DD0000001E6E30D0E64EC02F0150EF76E400ED6
:104DE000F66E5CEC02F0016A086AD3C226F0D2C209
:104DF00025F0D1C224F0D0C223F042EC01F0200E05
:104E000064EC02F0480E64EC02F07A0E64EC02F0FE
:104E10000D0E64EC02F0150EF76E4C0EF66E5CECA7
:104E200002F0016A086A30C319F02FC318F0A9EC28
:104E300000F0200E64EC02F0480E64EC02F07A0EF2
:104E400064EC02F00D0E64EC02F0150EF76E580ED5
:104E5000F66E5CEC02F0016A086A32C319F031C3E5
:104E600018F0A9EC00F0200E64EC02F0420E64ECA5
:104E700002F0640E64EC02F00D0E64EC02F0150E0C
:104E8000F76E600EF66E5CEC02F0016A03013351BE
:104E9000A6EC00F00D0E64EC02F0150EF76E6C0E31
:104EA000F66E5CEC02F0016A3451A6EC00F00D0ED7
:104EB00064EC02F0150EF76E780EF66E5CEC02F004
:104EC000016A3F51A6EC00F0200E64EC02F06D0E7A
:104ED00064EC02F0570E64EC02F00D0E64EC02F08C
:104EE000150EF76E840EF66E5CEC02F0016A355119
:104EF000A6EC00F0200E64EC02F0570E64EC02F019
:104F0000500E64EC02F04D0E64EC02F00D0E64ECF9
:104F100002F0150EF76E920EF66E5CEC02F0016A6E
:104F2000086AD9C219F0D8C218F0A4EC00F0200E1B
:104F300064EC02F0480E64EC02F07A0E64EC02F0CD
:104F40000D0E64EC02F03D510001E8A606D0540EAF
:104F500064EC02F0430E64EC02F0150EF76EA20E44
:104F6000F66E5CEC02F0016A086AD7C226F0D6C27F
:104F700025F0D5C224F0D4C223F042EC01F0200E7B
:104F800064EC02F0480E64EC02F07A0E64EC02F07D
:104F90000D0E64EC02F0890EF0EC02F00301406F9C
:104FA000150EF76EB20EF66E5CEC02F0A10E405DCF
:104FB000000109E3150EF76EBA0EF66E5CEC02F016
:104FC0000D0E64EC02F04B0E0301405D000102E2A5
:104FD000000E01D0010E3A6E640E0301405D010E19
:104FE000D8B0000E3A16000109E0150EF76EC20E99
:104FF000F66E5CEC02F00D0E64EC02F02A0E03017A
:10500000405D000109E2150EF76ECA0EF66E5CEC0B
:1050100002F00D0E64EC02F042EF2FF059EC2FF08D
:10502000F4C2D3F2F3C2D2F2F2C2D1F2F1C2D0F2A0
:10503000C00E0201D05DCB0ED159170ED259070E0A
:10504000D3590001D8B073D00201C06B150E020114
:10505000C05D00010EE200EEF1F00201C051EB5024
:105060000C6E0D0E0C5C000104E00201C02B00016F
:10507000EDE3090E0201C05D00010BE2300EF36E9C
:1050800000EEF1F00201C051F3CFEBFFC02B0001A5
:10509000F0D70D0EFA6F0201D36BD26BD16BD06BD0
:1050A000C06B090E0201C05D0001D8B040D0266A75
:1050B000256A246A0A0E236E26C013F025C012F05A
:1050C00024C011F023C010F0D3C21BF0D2C21AF0DA
:1050D000D1C219F0D0C218F05AEC04F013C026F077
:1050E00012C025F011C024F010C023F000EEF1F042
:1050F0000201C051EB500C6E2A6A296A286A0CC062
:1051000027F00F0E27142A6A296A286A276E23249B
:10511000D06F28502420D16F29502520D26F2A50DB
:105120002620D36F0201C02B0001D8A0BAD7070EEA
:105130000201D35D000114E311E1170E0201D25DFB
:1051400000010EE30BE1CB0E0201D15D000108E38B
:1051500005E1C00E0201D05D000102E3000E01D0A6
:10516000010E3A6E810E0201D05DD90ED1599F0E0B
:10517000D259380ED359000102E2000E01D0010EBF
:105180003A12D8A423EF2FF00201C06B0F0E0201D8
:10519000C05D00011AE200EEF1F00201C051EB50D7
:1051A00003011C6F0D0E1C5D00010FE0AA6A200EAA
:1051B0000201C025A96ED8B0AA2A03011C51F9EC3E
:1051C00002F00201C02B0001E1E3AA6A200E0201F5
:1051D000C025A96ED8B0AA2AFF0EF9EC02F0000192
:1051E000B9EC3FF042EF2FF059EC2FF0F4C2D7F2B8
:1051F000F3C2D6F2F2C2D5F2F1C2D4F2800E0201AD
:10520000D45D960ED559980ED659000ED759000187
:10521000D8B073D00201C06B150E0201C05D000151
:105220000EE200EEF1F00201C051EB500C6E0D0EDB
:105230000C5C000104E00201C02B0001EDE3080E4C
:105240000201C05D00010BE2300EF36E00EEF1F0E2
:105250000201C051F3CFEBFFC02B0001F0D70D0EC0
:10526000FA6F0201D76BD66BD56BD46BC06B090E8E
:105270000201C05D0001D8B040D0266A256A246AC8
:105280000A0E236E26C013F025C012F024C011F0C0
:1052900023C010F0D7C21BF0D6C21AF0D5C219F045
:1052A000D4C218F05AEC04F013C026F012C025F056
:1052B00011C024F010C023F000EEF1F00201C05143
:1052C000EB500C6E2A6A296A286A0CC027F00F0E70
:1052D00027142A6A296A286A276E2324D46F285043
:1052E0002420D56F29502520D66F2A502620D76F2D
:1052F0000201C02B0001D8A0BAD7000E0201D75D71
:10530000000114E311E1980E0201D65D00010EE3E5
:105310000BE1960E0201D55D000108E305E1800E68
:105320000201D45D000102E3000E01D0010E3A6ECD
:10533000C10E0201D45D0E0ED559160ED659020EBD
:10534000D759000102E2000E01D0010E3A12D8A492
:1053500023EF2FF0AA6A830EA96E0201D451F9EC53
:1053600002F0D551F9EC02F0D651F9EC02F0D75128
:10537000F9EC02F0000142EF2FF0DDEC2EF002011B
:10538000D96BD86B03012A930001F1510C6E2D0EDD
:105390000C5C02E103012A830201C06B0201C051CF
:1053A00003012AB3010F00EEF1F0EB500C6E0D0E6D
:1053B0000C5C000130E00201C05103012AB3010F6F
:1053C00000EEF1F0EB501C6F246A0A0E236E24C02D
:1053D00011F02350106E0201D803F3CF23F0F4CF65
:1053E00024F01150D803F35024261050D903F35061
:1053F00024261CC327F0286A27BE28680F0E27160C
:10540000000E281627502324D86F28502420D96F47
:10541000C02B0001C3D703012A510001E8A204D028
:105420000201D86DE86AD9570201D9AF06D0D00E73
:10543000D85D8A0ED959000102E3000E01D0010E99
:105440003A6E0201D9BF0AD0750ED95D07E300019B
:1054500007E1310E0201D85D000102E2000E01D029
:10546000010E3A120001D8A423EF2FF0AA6A870E8A
:10547000A96E0201D851F9EC02F0D951F9EC02F011
:10548000000129EC1CF042EF2FF059EC2FF0F2C292
:1054900030F3F1C22FF30201C06B0F0E0201C05DA9
:1054A00000011AE200EEF1F00201C051EB500301DD
:1054B0001C6F0D0E1C5D00010FE0AA6A300E020188
:1054C000C025A96ED8B0AA2A03011C51F9EC02F03C
:1054D0000201C02B0001E1E3AA6A300E0201C025DF
:1054E000A96ED8B0AA2AFF0EF9EC02F0000142EF33
:1054F0002FF059EC2FF0F2C232F3F1C231F3020176
:10550000C06B0F0E0201C05D000124E200EEF1F05D
:105510000201C051EB5003011C6F0D0E1C5D010E0A
:10552000D8A4000E3A6E2E0E1C5D010ED8A4000EFB
:105530003A1200010FE1AA6A400E0201C025A96ECD
:10554000D8B0AA2A03011C51F9EC02F00201C02BC9
:105550000001D7E3AA6A400E0201C025A96ED8B0A7
:10556000AA2AFF0EF9EC02F0000142EF2FF059ECED
:105570002FF0F1C233F3F15103011C6FAA6A500EF0
:10558000A96E1C51F9EC02F0000142EF2FF059EC2A
:105590002FF0F1C234F3010E0301345D00010DE17F
:1055A000AA6A510EA96E310EF9EC02F0AA6A520EE7
:1055B000A96EFF0EF9EC02F024D0020E0301345D57
:1055C00000010DE1AA6A510EA96E320EF9EC02F04B
:1055D000AA6A520EA96EFF0EF9EC02F012D0AA6A66
:1055E000510EA96E310EF9EC02F0AA6A520EA96EA4
:1055F000350EF9EC02F0AA6A530EA96EFF0EF9EC13
:1056000002F042EF2FF059EC2FF0F1C235F3020116
:10561000C06B0F0E0201C05D00011AE200EEF1F056
:105620000201C051EB5003011C6F0D0E1C5D000107
:105630000FE0AA6A700E0201C025A96ED8B0AA2A8E
:1056400003011C51F9EC02F00201C02B0001E1E35F
:10565000AA6A700E0201C025A96ED8B0AA2AFF0E50
:10566000F9EC02F0000142EF2FF0DDEC2EF017EC28
:105670001FF00201C06B0F0E0201C05D00011AE2B3
:1056800000EEF1F00201C051EB5003011C6F0D0E52
:105690001C5D00010FE0AA6A100E0201C025A96E70
:1056A000D8B0AA2A03011C51F9EC02F00201C02B68
:1056B0000001E1E3AA6A100E0201C025A96ED8B06C
:1056C000AA2AFF0EF9EC02F0000142EF2FF0DDEC08
:1056D0002EF017EC1FF00201C06B0F0E0201C05D2F
:1056E000000116E200EEF1F00201C051EB5003019F
:1056F0001C6F0D0E1C5D00010BE0AA6AC0C2A9FF61
:1057000003011C51F9EC02F00201C02B0001E5E39A
:10571000AA6AC0C2A9FFFF0EF9EC02F042EF2FF017
:1057200059EC2FF0F1C23FF303011E6B1D6B030117
:105730001E5300011FE10F0E03011D5D00011AE25F
:1057400000EEF1F003011D51EB501C6F0D0E1C5DBE
:10575000000110E0600E03011D25A96E000E1E2140
:10576000AA6E1C51F9EC02F003011D2B000E1E2342
:105770000001DDE3600E03011D25A96E000E1E2150
:10578000AA6EFF0EF9EC02F03F5142EC08F0CBECB0
:1057900004F034C02AF033C029F032C028F031C000
:1057A00027F0346A336A200E326E820E316E2AC0C0
:1057B00038F029C037F028C036F027C035F09BEC10
:1057C00007F034C024F333C023F332C022F331C0D6
:1057D00021F324C334F023C333F022C332F021C3B6
:1057E00031F09BEC06F01C6F150E1C5D000103E30D
:1057F000140E03011C6F03011C51040D1508000158
:1058000014E3F86A560EF324F66E1C0EF420F76EBD
:105810000900F5CF10F00900F5CF11F00900F5509F
:10582000090096EC03F010C0EBF2A8EC1BF042EF7D
:105830002FF0EFEC39F0150EF76ED40EF66E5CEC2F
:1058400002F0016A030139519FEC00F00D0E64EC87
:1058500002F0000142EF2FF00D0E64EC02F0150E85
:10586000F76EDE0EF66E5CEC02F0016A086A196AE9
:10587000040E186EA9EC00F02E0E64EC02F0010E7E
:10588000086E2D0EA7EC00F00D0E64EC02F042EF56
:105890002FF04F0E64EC02F04B0E64EC02F00D0E94
:1058A00064EC02F0010E156EF40E76EC03F0B1EC30
:1058B0002FF05AEF0FF09CEC33F0150EF76EF00E50
:1058C000F66E5CEC02F0016A16C326F015C325F0F3
:1058D00014C324F013C323F0020EE3EC00F0560EC1
:1058E00064EC02F0200E64EC02F064EC02F0150EA1
:1058F000F76EF80EF66E5CEC02F0016A0EC326F04D
:105900000DC325F00CC324F00BC323F0010EE3EC10
:1059100000F0430E64EC02F00D0E64EC02F042EF76
:105920002FF0140EF76E4E0EF66E5CEC02F00D0EBC
:1059300064EC02F093968A8672EC1BF0E3EC1BF0A9
:105940000B0E096EB80E026E37EC02F0F9E303019C
:105950001C6F440E1C5D010ED8A4000E3A6E640E3E
:105960001C5D010ED8A4000E3A12000114E00201E1
:10597000EB510001E8BE06D00201EB53000102E04A
:105980000201EB070001016A0201EB51A6EC00F0F5
:105990000D0E64EC02F0550E03011C5D010ED8A43F
:1059A000000E3A6E750E1C5D010ED8A4000E3A1260
:1059B000000112E00201EBBF04D07F0EEB5D00019D
:1059C00002E20201EB2B0001016A0201EB51A6EC9D
:1059D00000F00D0E64EC02F0450E03011C5D010E9B
:1059E000D8A4000E3A6E650E1C5D010ED8A4000E00
:1059F0003A12000103E0CFEC1BF044D2530E030136
:105A00001C5D010ED8A4000E3A6E730E1C5D010ED3
:105A1000D8A4000E3A1200010BE0CFEC1BF0AA6AEA
:105A2000600EA96E0201EB51F9EC02F000012AD2DE
:105A3000A8EC1BF085D7C1D917EC1FF003012A9100
:105A40000001F1510C6E4F0E0C5C010ED8A4000E3B
:105A50003A6EF2510C6E4E0E0C5C010ED8A4000E84
:105A60003A1604E003012A83000152D0F1510C6E72
:105A7000590E0C5C010ED8A4000E3A6EF2510C6E59
:105A8000450E0C5C010ED8A4000E3A16F3510C6EB4
:105A9000530E0C5C010ED8A4000E3A1604E003016C
:105AA0002A83000135D0F1510C6E4F0E0C5C010EB3
:105AB000D8A4000E3A6EF2510C6E460E0C5C010E2C
:105AC000D8A4000E3A16F3510C6E460E0C5C010E73
:105AD000D8A4000E3A1604E003012A93000118D05E
:105AE000F1510C6E4E0E0C5C010ED8A4000E3A6EF5
:105AF000F2510C6E4F0E0C5C010ED8A4000E3A163B
:105B000004E003012A93000102D003012A8100016D
:105B100012000D0E64EC02F0160EF76E000EF66E1B
:105B20005CEC02F00D0E64EC02F00D0E64EC02F081
:105B3000160EF76E1A0EF66E5CEC02F00D0E64ECAB
:105B400002F0160EF76E380EF66E5CEC02F00D0EDB
:105B500064EC02F0160EF76E580EF66E5CEC02F076
:105B60000D0E64EC02F0160EF76E700EF66E5CEC25
:105B700002F00D0E64EC02F0160EF76E8A0EF66E51
:105B80005CEC02F00D0E64EC02F0160EF76EAE0E39
:105B9000F66E5CEC02F00D0E64EC02F0160EF76E81
:105BA000F00EF66E5CEC02F00D0E64EC02F0170ED7
:105BB000F76E0A0EF66E5CEC02F00D0E64EC02F06D
:105BC000170EF76E400EF66E5CEC02F00D0E64ECF4
:105BD00002F0170EF76E5A0EF66E5CEC02F00D0E28
:105BE00064EC02F0170EF76E820EF66E5CEC02F0BB
:105BF0000D0E64EC02F0170EF76E9E0EF66E5CEC66
:105C000002F00D0E64EC02F0170EF76EC40EF66E85
:105C10005CEC02F00D0E64EC02F0170EF76EF20E63
:105C2000F66E5CEC02F00D0E64EC02F0180EF76EEE
:105C3000180EF66E5CEC02F00D0E64EC02F0180E1D
:105C4000F76E480EF66E5CEC02F00D0E64EC02F09E
:105C5000180EF76E7E0EF66E5CEC02F00D0E64EC24
:105C600002F0180EF76EAA0EF66E5CEC02F00D0E46
:105C700064EC02F0180EF76ED40EF66E5CEC02F0D7
:105C80000D0E64EC02F0180EF76EFE0EF66E5CEC74
:105C900002F00D0E64EC02F0190EF76E2C0EF66E8B
:105CA0005CEC02F00D0E64EC02F0190EF76E5A0E69
:105CB000F66E5CEC02F00D0E64EC02F0190EF76E5D
:105CC000820EF66E5CEC02F00D0E64EC02F0190E22
:105CD000F76EA80EF66E5CEC02F00D0E64EC02F0AE
:105CE000190EF76ECA0EF66E5CEC02F00D0E64EC47
:105CF00002F0190EF76EF60EF66E5CEC02F00D0E69
:105D000064EC02F01A0EF76E260EF66E5CEC02F0F2
:105D10000D0E64EC02F01A0EF76E560EF66E5CEC89
:105D200002F00D0E64EC02F01A0EF76E7C0EF66EA9
:105D30005CEC02F00D0E64EC02F01A0EF76EBC0E75
:105D4000F66E5CEC02F00D0E64EC02F01A0EF76ECB
:105D5000F20EF66E5CEC02F00D0E64EC02F01B0E1F
:105D6000F76E200EF66E5CEC02F00D0E64EC02F0A5
:105D70001B0EF76E5A0EF66E5CEC02F00D0E64EC24
:105D800002F01B0EF76E7A0EF66E5CEC02F00D0E52
:105D900064EC02F01B0EF76EA00EF66E5CEC02F0E7
:105DA0000D0E64EC02F01B0EF76EBA0EF66E5CEC94
:105DB00002F00D0E64EC02F065D003012A95020199
:105DC000C06B000100EEF1F00201C051EB500C6E0F
:105DD000200E0C5CD8A4010E3A6EFD0EC05D010EC3
:105DE000D8B0000E3A16000112E000EEF1F0020108
:105DF000C051EB500C6E0D0E0C5C000104E1030170
:105E00002A85000112000201C02B0001DAD702012D
:105E1000C02BC051FF080B6ECD6B0201CD510B5C46
:105E2000000110E30201CD51C02500EEF1F0EBCFEF
:105E30000CF000EEF1F0CD510CC0EBFF0201CD2BC8
:105E40000001EBE31200450E64EC02F0520E64EC2C
:105E500002F064EC02F04F0E64EC02F0520E64ECBF
:105E600002F00D0E64EC02F0630E64EC02F06D0EB5
:105E700064EC02F0640E64EC02F03E0E64EC02F09E
:105E8000A6EF1EF04F0E64EC02F04B0E64EC02F035
:105E90000D0E64EC02F0630E64EC02F06D0E64EC27
:105EA00002F0640E64EC02F03E0E64EC02F0A6EF29
:105EB0001EF083DF010E0201C06F0001F1510C6E74
:105EC0000F0B0201F46BF36BF26BF16F000100EE4C
:105ED000F1F00201C051EB500C6E0D0E0C5C000194
:105EE000D8B43ED0266A256A246A0A0E236E26C0DC
:105EF00013F025C012F024C011F023C010F0F4C23A
:105F00001BF0F3C21AF0F2C219F0F1C218F05AEC09
:105F100004F013C026F012C025F011C024F010C008
:105F200023F000EEF1F00201C051EB500C6E2A6A32
:105F3000296A286A0CC027F00F0E27142A6A296ADA
:105F4000286A276E2324F16F28502420F26F2950ED
:105F50002520F36F2A502620F46FC02B0001B6D7FE
:105F6000120003011E6B1D6B1EC3AAFF1DC3A9FFF8
:105F7000F2EC02F01C6F03011C29000112E002EE9A
:105F800077F003011D511CC3EBFF1D2B000E1E23D8
:105F90001EC3AAFF1DC3A9FFF2EC02F01C6F000193
:105FA000EAD7F36A02EE77F003011D51F3CFEBFF5E
:105FB000200EF0EC02F01C6F1C2900010BE1190E01
:105FC0000201D36FEA0ED26F850ED16F800ED06FB3
:105FD000000182D00201D36BD26BD16BD06BC06B4E
:105FE00003011C290001D8B443D0266A256A246A1B
:105FF0000A0E236E26C013F025C012F024C011F043
:1060000023C010F0D3C21BF0D2C21AF0D1C219F0D3
:10601000D0C218F05AEC04F013C026F012C025F0DC
:1060200011C024F010C023F02A6A296A286A1CC310
:1060300027F00F0E27142A6A296A286A276E23245C
:106040000201D06F28502420D16F29502520D26F13
:106050002A502620D36FC02BAA6A200EC025A96E15
:10606000D8B0AA2AF2EC02F003011C6F0001B8D7E5
:10607000070E0201D35D000114E311E1170E0201C6
:10608000D25D00010EE30BE1CB0E0201D15D0001F8
:1060900008E305E1C00E0201D05D000102E3000E3D
:1060A00001D0010E3A6E810E0201D05DD90ED15998
:1060B0009F0ED259380ED359000102E2000E01D0D2
:1060C000010E3A1209E0190E0201D36FEA0ED26FE7
:1060D000850ED16F800ED06F0301306B2F6B300EA9
:1060E000F0EC02F01C6F1C29000107E1030E030114
:1060F000306F7A0E2F6F000136D00201C06B0301A2
:106100001C29000130E0246A0A0E236E24C019F015
:106110002350186E03012F03F3CF23F0F4CF24F0A4
:1061200019502F03F350242618503003F35024261F
:10613000286A1CC327F00F0E2716000E28162750BA
:1061400023242F6F28502420306F0201C02BAA6A0D
:10615000300EC025A96ED8B0AA2AF2EC02F00301D5
:106160001C6F0001CCD70301326B316B400EF0EC99
:1061700002F01C6F1C29000107E1270E0201F86FD5
:10618000100EF76F000173D00201C06B03011C29D0
:10619000000130E0246A0A0E236E24C019F0235057
:1061A000186E03013103F3CF23F0F4CF24F019501C
:1061B0003103F350242618503203F3502426286A62
:1061C0001CC327F00F0E2716000E28162750232475
:1061D000316F28502420326F0201C02BAA6A400E72
:1061E000C025A96ED8B0AA2AF2EC02F003011C6FF8
:1061F0000001CCD703013253000109E12D0E030148
:10620000315D000104E20301326B2D0E316F050E8A
:106210000301325D00010BE305E1DD0E0301315D99
:10622000000105E3050E0301326FDC0E316F03013F
:1062300031512D0A3211000107E1560E0201F86FAB
:10624000CE0EF76F000113D0136A0F0E126E420EBE
:10625000116E400E106E31C318F032C319F01A6A75
:106260001B6A15EC04F011C0F8F210C0F7F2500EE2
:10627000F0EC02F00301336F3329000105E1070E52
:106280000301336F000103D00F0E03013317070E14
:106290000301335DD8A4010E3A6E080E335DD8A415
:1062A000010E3A16000103E0080E0301336F0001EE
:1062B000AA6A510EA96EF2EC02F003011C6F1C29B0
:1062C000000108E1D8900201F735F96FF835FA6F4F
:1062D000000166D00F0E03011C150201C06FAA6AEF
:1062E000520EA96EF2EC02F003011C6F1C29000192
:1062F00019E0246A0A0E236E24C010F00201C05176
:106300002302F3CF23F0F4CF24F01002F35024261D
:10631000286A1CC327F00F0E2716000E28162350DC
:106320002724C06F010E0201C05DD8A4010E3A6E91
:10633000020EC05DD8A4010E3A160F0EC05DD8A49F
:10634000010E3A16000103E0010E0201C06F0001C8
:10635000C0C234F30F0E0201C05D000116E1F7C2A6
:1063600031F0F8C232F044EC08F0386A376A400E77
:10637000366E7F0E356E9BEC07F0E9EC07F00201FC
:10638000F96F32C0FAF200010AD00201C051F703DE
:10639000F3CFF9F2F4CFFAF2F803F350FA27000141
:1063A000600EF0EC02F003011C6F1C29000105E1F6
:1063B0000A0E03013F6F00012FD003013F6B020162
:1063C000C06B03011C29000127E0246A0A0E236E1A
:1063D00024C010F003013F512302F3CF23F0F4CF88
:1063E00024F01002F3502426286A1CC327F00F0E55
:1063F0002716000E2816235027243F6F0201C02BBA
:10640000AA6A600EC025A96ED8B0AA2AF2EC02F0E2
:1064100003011C6F0001D5D703013F5142EC08F086
:10642000CBEC04F034C02AF033C029F032C028F09D
:1064300031C027F0346A336A200E326E820E316E1C
:106440002AC038F029C037F028C036F027C035F010
:106450009BEC07F034C024F333C023F332C022F3A3
:1064600031C021F324C334F023C333F022C332F00C
:1064700021C331F09BEC06F01C6F150E1C5D000172
:1064800003E3140E03011C6F03011C51040D1508D6
:10649000000114E3F86AAE0EF324F66E1C0EF4202D
:1064A000F76E0900F5CF10F00900F5CF11F00900E3
:1064B000F550090096EC03F010C0EBF2030E030157
:1064C0001C27150E1C5D000103E3140E03011C6F55
:1064D00003011C51040D1508000114E3F86A060EAF
:1064E000F324F66E1D0EF420F76E0900F5CF10F0C0
:1064F0000900F5CF11F00900F550090096EC03F002
:1065000010C036F3250E0301286F700EF0EC02F078
:106510001C6F1C290001D8B44BD00201C06B0301D1
:10652000356B03011C29000127E0246A0A0E236E43
:1065300024C010F0030135512302F3CF23F0F4CF30
:1065400024F01002F3502426286A1CC327F00F0EF3
:106550002716000E281623502724356F0201C02B62
:10656000AA6A700EC025A96ED8B0AA2AF2EC02F071
:1065700003011C6F0001D5D7140E0301355D000126
:1065800003E2140E0301356F790E0301355D00013E
:1065900003E3780E0301356F00010B0E116EB80E88
:1065A000106E156A35C314F043EC04F00301286F34
:1065B0000001830EF0EC02F00201D46FF2EC02F065
:1065C000D56FF2EC02F0D66FF2EC02F0D76F000E4E
:1065D000D75D000114E311E1980E0201D65D0001C0
:1065E0000EE30BE1960E0201D55D000108E305E123
:1065F000800E0201D45D000102E3000E01D0010E05
:106600003A6E410E0201D45D8A0ED559F70ED65965
:10661000010ED759000102E2000E01D0010E3A121C
:1066200009E0010E0201D76FC90ED66FC30ED56FF8
:10663000800ED46F0001870EF0EC02F00201D86FDB
:10664000F2EC02F0D96FD9AF06D0D00ED85D8A0E29
:10665000D959000102E3000E01D0010E3A6E020189
:10666000D9BF0AD0750ED95D07E3000107E1310EED
:106670000201D85D000102E2000E01D0010E3A12C3
:10668000000105E0040E0201D96FB00ED86F0001C1
:10669000820EF0EC02F003013E6F800EF0EC02F08F
:1066A0003C6F810EF0EC02F03D6F890EF0EC02F0D1
:1066B000406F8A0EF0EC02F00201EC6F8B0EF0ECF2
:1066C00002F09B6E03012A97296B01EEDEF0EF6A60
:1066D00001EEEEF0EF6A01EEFEF0EF6A300E02011D
:1066E000BB6F02EE3EF0EF6A03013A6B02EE0EF072
:1066F000EE6E2E0EEE6E300EEE6EEF6A02EE1EF0B5
:10670000EF6A02EE2EF0EF6A0201FC6BFB6B9BCF8F
:1067100039F30301D89239BBD882D8B2398DD8A2C7
:10672000399DD89239BBD882D8B2398FD8A2399F37
:10673000960E2E6F00011200010E0201896F8A6F02
:10674000080E8B6F000167EC3FF01B0EF76EDE0E3C
:10675000F66E5CEC02F0016A02018951A6EC00F0D1
:106760000D0E64EC02F01B0EF76EEE0EF66E5CEC96
:1067700002F0016A020E086E8A518AEC00F0020EE5
:10678000086E8B518AEC00F00D0E64EC02F01B0ECB
:10679000F76EF80EF66E5CEC02F0016A020E086EFF
:1067A0008C518AEC00F00D0E64EC02F01C0EF76EBA
:1067B000080EF66E5CEC02F0016A020E086E8D5156
:1067C0008AEC00F0020E086E8E518AEC00F00D0E7D
:1067D00064EC02F01C0EF76E1C0EF66E5CEC02F020
:1067E000016A020E086E8F518AEC00F00D0E64EC07
:1067F00002F01C0EF76E2C0EF66E5CEC02F0016AD5
:10680000020E086E90518AEC00F00D0E64EC02F05E
:10681000030E0201896F140E8A6F180E8B6F8C6B3A
:10682000060E8D6F000167EC3FF002018B510301F2
:106830001E6F02018C5103011D6F1DC331F01EC379
:1068400032F044EC08F0386A376A400E366E800E3B
:10685000356E9BEC07F034C026F033C025F032C013
:1068600024F031C023F0386A376A200E366E890E64
:10687000356E26C034F025C033F024C032F023C07A
:1068800031F035EC07F034C016F333C015F332C0E5
:1068900014F331C013F302018D5103011E6F020185
:1068A0008E5103011D6F246BC00E236F600E226F8B
:1068B0007C0E216F1DC331F01EC332F044EC08F092
:1068C00024C338F023C337F022C336F021C335F098
:1068D0009BEC07F034C026F033C025F032C024F022
:1068E00031C023F0386A800E376E120E366E870E76
:1068F000356E26C034F025C033F024C032F023C0FA
:1069000031F0A5EC06F034C00EF333C00DF332C005
:106910000CF331C00BF3000112000301206B1F6B5D
:106920000201C06B0A0E0201C05D00010FE2010E00
:1069300008EC03F00C6E24C00DF00C5003011F276F
:106940000D5020230201C02B0001ECE31FC331F0E6
:1069500020C332F044EC08F0386A400E376E1C0E4B
:10696000366E8A0E356EA5EC06F034C026F033C0C4
:1069700025F032C024F031C023F0386A376A480E5F
:10698000366E840E356E26C034F025C033F024C038
:1069900032F023C031F035EC07F034C00AF333C0D5
:1069A00009F332C008F331C007F312000301206B72
:1069B0001F6B0201C06B0A0E0201C05D00010FE2F5
:1069C000000E08EC03F00C6E24C00DF00C50030117
:1069D0001F270D5020230201C02B0001ECE31FC331
:1069E00031F020C332F044EC08F0386A400E376EC4
:1069F0001C0E366E8A0E356EA5EC06F034C026F0FD
:106A000033C025F032C024F031C023F0386A376A31
:106A1000480E366E840E356E26C034F025C033F035
:106A200024C032F023C031F035EC07F034C012F34B
:106A300033C011F332C010F331C00FF31200030161
:106A4000206B1F6B0201C06B0A0E0201C05D0001CA
:106A50000FE2030E08EC03F00C6E24C00DF00C5096
:106A600003011F270D5020230201C02B0001ECE37E
:106A7000386A400E376E1C0E366E8B0E356E20C394
:106A800032F01FC331F044EC08F035EC07F034C0AD
:106A900000F333C0FFF232C0FEF231C0FDF212004B
:106AA0000301206B1F6B0201C06B0A0E0201C05D67
:106AB00000010FE20F0E08EC03F00C6E24C00DF085
:106AC0000C5003011F270D5020230201C02B000191
:106AD000ECE3386A400E376E1C0E366E8B0E356E48
:106AE00020C332F01FC331F044EC08F035EC07F05E
:106AF00034C004F333C003F332C002F331C001F3F6
:106B000012000301206B1F6B1E6B1D6B0201C06B1B
:106B10000A0E0201C05D000119E2040E08EC03F048
:106B20000C6E24C00DF00C5003011F270D502023C4
:106B30000F0E08EC03F00C6E24C00DF00C501D2756
:106B40000D501E230201C02B0001E2E3386A400E03
:106B5000376E1C0E366E8B0E356E1EC332F01DC3A3
:106B600031F044EC08F035EC07F034C004F333C0E6
:106B700003F332C002F331C001F31EC324F01DC37E
:106B800023F003011F51235C236E20512458246EEF
:106B900024C011F023C010F0156A050E146E43ECEA
:106BA00004F0236E11C024F023503EA1E86A056F63
:106BB00024503EA1E86A066F00011200D76AD66A27
:106BC00003011E6B1D6B2A8382A02A93320E75EC83
:106BD00003F00001E86A03012AB3010F82B0010843
:106BE00000012CE103011D2B000E1E23320E75EC5B
:106BF00003F0020E1E5D000120E305E1590E0301C2
:106C00001D5D00011AE301EE47F00D0EEE6E0A0E57
:106C1000EE6E1C0EF76E380EF66EBAEC04F00D0E2A
:106C2000EE6E0A0EEE6EEF6A00010CEC1DF0270E00
:106C3000156E100E76EC03F0C1D7CBD782B0FED71D
:106C400082A0FED7D58E82B0FED782A0FED7D59E79
:106C5000D6CF18F3D7CF19F3F40E0301195DBA0E8E
:106C6000D8B4185D000102E20301392BF50E0301CF
:106C7000195D000108E305E11F0E0301185D000125
:106C800002E3030139073F0E030139159B6EF40E31
:106C9000195DBA0ED8B4185D000102E2000E01D0F1
:106CA000010E3A6EF50E0301195D000108E305E1DE
:106CB0001F0E0301185D000102E3000E01D0010E5A
:106CC0003A16000110E0AA6A8B0EA96E9B50F9ECEF
:106CD00002F003013E8FAA6A820EA96E3E51F9ECC2
:106CE00002F00001120001EE47F0200EEE6EEE6E93
:106CF000020E016E086A19C319F018C318F0A9EC46
:106D000000F0200EEE6EEE6E020E016E03013951A0
:106D10009FEC00F00D0EEE6EEF6A00010CEC1DF022
:106D2000030E156EE80E76EC03F0D76AD66A86D7A6
:106D300094988B8803013D3500011CE2800E026EA1
:106D4000400E096E206A40C31FF0066A056A200ED5
:106D5000016E120EF76E120EF66E0900F55003E08A
:106D6000C5EC01F0FAD70D0EC5EC01F00A0EC5EC2A
:106D700001F03BD0800E026E400E096E206A40C3C7
:106D80001FF0066A056A200E016EB50EC5EC01F013
:106D9000620EC5EC01F0060EC5EC01F0570EC5EC15
:106DA00001F0080EC5EC01F0000EC5EC01F0010E7B
:106DB000C5EC01F0000EC5EC01F0000EC5EC01F0D1
:106DC000000EC5EC01F0500EC5EC01F04F0EC5EC05
:106DD00001F0540EC5EC01F0530EC5EC01F0AC0E01
:106DE000C5EC01F0850EC5EC01F0A20ED36ED28881
:106DF000C290719E020E156E710E76EC03F0D29861
:106E0000D20ED36EC280718E94988B9803013D355B
:106E100000011CE2800E026E400E096E206A40C323
:106E20001FF0066A056A200E016E120EF76E200E24
:106E3000F66E0900F55003E0C5EC01F0FAD70D0E2F
:106E4000C5EC01F00A0EC5EC01F03BD0800E026EDD
:106E5000400E096E206A40C31FF0066A056A200EC4
:106E6000016EB50EC5EC01F0620EC5EC01F0060E28
:106E7000C5EC01F0570EC5EC01F0080EC5EC01F0B1
:106E8000000EC5EC01F0010EC5EC01F0000EC5ECE2
:106E900001F0000EC5EC01F0000EC5EC01F0200E73
:106EA000C5EC01F04E0EC5EC01F0550EC5EC01F03D
:106EB000520EC5EC01F07B0EC5EC01F0C30EC5EC23
:106EC00001F0130E156E880E76EC03F0096A010EC0
:106ED000026E37EC02F0D8A02BD703011C6F450ED1
:106EE0001C5D010ED8A4000E3A6E650E1C5D010EED
:106EF000D8A4000E3A12000104E0CEEC1DF042EFDF
:106F00002FF016D700EEF1F0240EEE6E470EEE6E67
:106F1000EF6A40C325F3800E026E800E096E206A70
:106F200040C31FF00B0E066EB80E056E84EC01F028
:106F300038E32408FBE184EC01F033E303011C6F28
:106F4000020E0201C06F510E0201C05D00011AE283
:106F5000800E026E800E096E206A40C31FF0A1EC05
:106F600001F003011C6F00EEF1F00201C0511CC3DF
:106F7000EBFF0D0E03011C5D000104E00201C02BBC
:106F80000001E1E30201C029F10FE96E000EEA6A97
:106F9000EA22EF6A016A560E076E196AF10E74EC66
:106FA00001F00001030E096EE80E026E37EC02F0EC
:106FB000D8A0A8D703011C6F550E1C5D010ED8A4E4
:106FC000000E3A6E750E1C5D010ED8A4000E3A122A
:106FD000000109E00301402B016A4051A6EC00F0DA
:106FE0000D0E64EC02F0440E03011C5D010ED8A4EA
:106FF000000E3A6E640E1C5D010ED8A4000E3A120B
:10700000000109E003014007016A4051A6EC00F0CD
:107010000D0E64EC02F0530E03011C5D010ED8A4AA
:10702000000E3A6E730E1C5D010ED8A4000E3A12CB
:1070300000010AE0AA6A890EA96E03014051F9EC29
:1070400002F0000142EF2FF0450E03011C5D010E1E
:10705000D8A4000E3A6E650E1C5D010ED8A4000E79
:107060003A12000104E025C340F342EF2FF04AD763
:107070008DEC34F01FEC35F0F2EC1BF008EC34F042
:1070800001EE47F0240EEE6EEE6EEE6EEE6E12EE38
:1070900077F0110EE75204E0E6CFEEFFE82EFAD7C4
:1070A0002C0EEE6E020E016E0EC326F00DC325F0FF
:1070B0000CC324F00BC323F0010EE3EC00F02C0E04
:1070C000EE6E020E016E0AC326F009C325F008C356
:1070D00024F007C323F0010EE3EC00F02C0EEE6E5B
:1070E000020E016E16C326F015C325F014C324F05A
:1070F00013C323F0E3EC00F02C0EEE6E020E016ED3
:1071000000C326F0FFC225F0FEC224F0FDC223F02A
:10711000E3EC00F0EF6A03011B6B01EE47F0E86A55
:10712000EE5202E0E83EFCD70B6E040E0201CD6F7A
:107130000201CD510B5C00010FE301EE47F00201AB
:10714000CD51E926000EEA22EF500C6E03011B1B05
:107150000201CD2B0001ECE301EE47F0EE50FEE121
:10716000ED522A0EEE6E020E016E086E03011B51E7
:107170008AEC00F00D0EEE6E0A0EEE6EEF6A000164
:107180000CEC1DF0130E096E880E026E37EC02F047
:10719000D8A06ED703011C6F450E1C5D010ED8A44C
:1071A000000E3A6E650E1C5D010ED8A4000E3A1258
:1071B0000001D8A442EF2FF05BD7B6EC1CF0016AB7
:1071C000086ADFC226F0DEC225F0DDC224F0DCC290
:1071D00023F041EC01F00D0E64EC02F0FCEC1BF02E
:1071E000020E0201896F220E8A6F8B6B080E8C6F64
:1071F000000167EC3FF01C0EF76E4E0EF66E5CEC75
:1072000002F0016A02018B51A6EC00F0200E64EC42
:1072100002F08C51A6EC00F0200E64EC02F08D51CF
:10722000A6EC00F0200E64EC02F08E51A6EC00F00B
:107230000D0E64EC02F0030E096EE80E026E37ECE0
:1072400002F00001CDE303011C6F450E1C5D010E31
:10725000D8A4000E3A6E650E1C5D010ED8A4000E77
:107260003A120001D8A442EF2FF0BAD7949A8B9A21
:10727000820E026E400E096E810E036E010E046EC8
:107280000A6E120E106E4AEC03F0400E106E4AECBD
:1072900003F0080E106E4AEC03F0106A4AEC03F09B
:1072A000949A8B8A81A2FED7949A8B9A820E026E50
:1072B000400E096E810E036E010E046E0A6E440EBE
:1072C000106E4AEC03F0820E026E800E096E810E83
:1072D000036E010E046E0A6A1EEC03F010C01CF36C
:1072E00003011C29000108E0949A8B8A010E75ECB9
:1072F00003F0949A8B9ADAD7820E026E800E096E92
:10730000810E036E010E046E0A6A1EEC03F010C0BB
:1073100041F31EEC03F010C042F31EEC03F010C06A
:1073200043F31EEC03F010C044F31EEC03F010C056
:1073300045F31EEC03F010C046F31EEC03F010C042
:1073400047F31EEC03F010C048F3949A8B8A016A4D
:10735000020E086E030141518AEC00F0200E64EC2D
:1073600002F0020E086E42518AEC00F0200E64EC2E
:1073700002F0020E086E43518AEC00F0200E64EC1D
:1073800002F0020E086E44518AEC00F0200E64EC0C
:1073900002F0020E086E45518AEC00F0200E64ECFB
:1073A00002F0020E086E46518AEC00F0200E64ECEA
:1073B00002F0020E086E47518AEC00F0200E64ECD9
:1073C00002F0020E086E48518AEC00F0200E64ECC8
:1073D00002F00D0E64EC02F0000142EF2FF0D76ACC
:1073E000D66A82B0FED782A0FED7D58E82B0FED7F5
:1073F00082A0FED7D59ED6CF18F3D7CF19F3F40EBF
:107400000301195D000106E307E1A70E0301185D02
:10741000000102E20301392BF50E0301195D0001A1
:1074200008E305E13C0E0301185D000102E30301DE
:107430003907F40E0301195D000106E307E1A70E09
:107440000301185D000102E2000E01D0010E3A6E48
:10745000F50E0301195D000108E305E13C0E03018F
:10746000185D000102E3000E01D0010E3A16000182
:10747000D8A412003F0E030139159B6E140E75EC53
:1074800003F00001ACD70201CD6B000173EC1DF0DD
:10749000246A0A0E236E020144510C6E286A0CC045
:1074A00027F00F0E2716000E281624C019F02350BF
:1074B000186E2702F3CF23F0F4CF24F019502702DF
:1074C000F350242618502802F350242645510E6EFE
:1074D000286A0EC027F00F0E2716000E281623501C
:1074E00027240301516F246A0A0E236E02014651BC
:1074F0000C6E286A0CC027F00F0E2716000E2816F7
:1075000024C019F02350186E2702F3CF23F0F4CFD4
:1075100024F019502702F350242618502802F35063
:10752000242647510E6E286A0EC027F00F0E27162C
:10753000000E2816235027240301526F386A376A39
:10754000700E366E840E356E525142EC08F035ECFA
:1075500007F034C026F033C025F032C024F031C02B
:1075600023F0515142EC08F026C038F025C037F026
:1075700024C036F023C035F0A7EC06F034C024F365
:1075800033C023F332C022F331C021F3246A0A0E40
:10759000236E020149510C6E286A0CC027F00F0EB1
:1075A0002716000E281624C019F02350186E270243
:1075B000F3CF23F0F4CF24F019502702F350242600
:1075C00018502802F35024264A510E6E286A0EC025
:1075D00027F00F0E2716000E28162350272403012C
:1075E000566F0201CD6B000172EC1DF002EE44F00B
:1075F000EECFF3FFEFCFF4FFF3504E0AF41005E1A6
:107600005A0E03015127000115D0030151515A08A8
:10761000516F525300010EE00301510752513C08D3
:10762000526F5653000105E003015207565164089A
:10763000566F0001D89003015237D8905637020197
:10764000CD6B000171EC1DF0246A640E236E020103
:1076500044510C6E286A0CC027F00F0E2716000E3E
:10766000281624C019F02350186E2702F3CF23F0F8
:10767000F4CF24F019502702F35024261850280282
:10768000F3502426286A0A0E276E45510E6E2C6A86
:107690000EC02BF00F0E2B16000E2C1628C019F062
:1076A0002750186E2B02F3CF27F0F4CF28F0195093
:1076B0002B02F350282618502C02F350282627506E
:1076C00023262850242246510F6E286A0FC027F027
:1076D0000F0E2716000E2816275023240301536F80
:1076E00028502420546F246A0A0E236E0201475149
:1076F0000C6E286A0CC027F00F0E2716000E2816F5
:1077000024C019F02350186E2702F3CF23F0F4CFD2
:1077100024F019502702F350242618502802F35061
:10772000242648510E6E286A0EC027F00F0E271629
:10773000000E2816235027240301556F386A376A34
:10774000700E366E840E356E555142EC08F035ECF5
:1077500007F034C026F033C025F032C024F031C029
:1077600023F053C331F054C332F044EC08F026C088
:1077700038F025C037F024C036F023C035F0A7EC30
:1077800006F034C024F333C023F332C022F331C0F7
:1077900021F3246A0A0E236E02014A510C6E286AF4
:1077A0000CC027F00F0E2716000E281624C019F063
:1077B0002350186E2702F3CF23F0F4CF24F0195092
:1077C0002702F350242618502802F35024264B5148
:1077D0000E6E286A0EC027F00F0E2716000E281610
:1077E000235027240301576F0201CD6B000170EC79
:1077F0001DF002EE44F0EECFF3FFEFCFF4FFF350B5
:10780000450AF41007E1B40E03015327000E542378
:1078100000011AD003015351B408536F000E5455A0
:10782000546F5553000110E003015307000E545BE1
:1078300055513C08556F5753000105E003015507AA
:1078400057516408576F000102EE44F0EF6A54C3C9
:1078500011F053C310F0156A140E146E43EC04F0CB
:10786000236E11C024F0410E232403011C6F02EE8D
:1078700044F0EE50FEE1ED521CC3EEFFEF6A51C33F
:1078800010F00A0E40EC04F0236E246A410E23240B
:107890001C6F02EE44F0EE50FEE1ED521CC3EEFF11
:1078A000EF6A246A300E236E54C328F053C327F0C6
:1078B00028C011F027C010F0156A140E146E43ECA6
:1078C00004F019C028F018C027F0D89028322732C9
:1078D000235027241C6F02EE44F0EE50FEE1ED52DF
:1078E0001CC3EEFFEF6A116A51C310F0156A0A0E4D
:1078F000146E43EC04F019C024F018C023F0300ECD
:1079000023241C6F02EE44F0EE50FEE1ED521CC346
:10791000EEFFEF6A246A410E236E000E53B1010E92
:10792000286A276E28503C0DF3CF28F027503C0DD5
:10793000F3CF27F0F450282655512726000E282291
:1079400028C011F027C010F0156A050E146E43EC24
:1079500004F0276E11C028F0235027241C6F02EE7C
:1079600044F0EE50FEE1ED521CC3EEFFEF6A52C34D
:1079700010F0050E40EC04F0236E246A410E23241F
:107980001C6F02EE44F0EE50FEE1ED521CC3EEFF20
:10799000EF6A000E3DBB010E3A6E000E2AB7010ED3
:1079A0003A120001D8B4DFD03C0E030153A1000EFF
:1079B000236E53A1000E246E555123241D6F000E1B
:1079C00024201E6F1EC311F01DC310F0156A050E92
:1079D000146E43EC04F018C01CF31C51640DF3CF7B
:1079E00023F0F4CF24F0575123241D6F000E2420E0
:1079F0001E6F1EC311F01DC310F0156A320E146EF7
:107A000043EC04F0236E11C024F0300E23241C6FCD
:107A100002EE44F0EE50FEE1ED521CC3EEFFEF6AC1
:107A20001EC311F01DC310F0156A320E146E43EC24
:107A300004F018C057F3116A52C310F0156A050E0E
:107A4000146E43EC04F018C01CF31C51640DF3CF0A
:107A500023F0F4CF24F0565123241D6F000E242070
:107A60001E6F1EC311F01DC310F0156A320E146E86
:107A700043EC04F0236E11C024F0300E23241C6F5D
:107A80001EC311F01DC310F0156A320E146E43ECC4
:107A900004F018C056F302EE44F0EE50FEE1ED5251
:107AA0001CC3EEFFEF6ADF0E386E4F0E376E050E09
:107AB000366E800E356E575142EC08F035EC07F00B
:107AC00034C026F033C025F032C024F031C023F09A
:107AD000346A336A020E326E850E316E26C038F07B
:107AE00025C037F024C036F023C035F0A7EC06F0EF
:107AF000E9EC07F01C6F02EE44F0EE50FEE1ED52AF
:107B00001CC3EEFFEF6ADF0E386E4F0E376E050EA8
:107B1000366E800E356E565142EC08F035EC07F0AB
:107B200034C026F033C025F032C024F031C023F039
:107B3000346A336A020E326E850E316E26C038F01A
:107B400025C037F024C036F023C035F0A7EC06F08E
:107B5000E9EC07F01C6F02EE44F0EE50FEE1ED524E
:107B60001CC3EEFFEF6A0001120003013D5100014A
:107B7000E8A601D012008DEC34F0346A336AC00EEE
:107B8000326E7F0E316E0AC338F009C337F008C376
:107B900036F007C335F023EC06F00108D8B46AD0FC
:107BA0000AC338F009C337F008C336F007C335F00D
:107BB000660E346E336E4E0E326E830E316EA5EC51
:107BC00006F034C026F033C025F032C024F031C0B6
:107BD00023F0346A336A2A0E326E850E316E26C067
:107BE00038F025C037F024C036F023C035F09BECC8
:107BF00007F034C024F333C023F332C022F331C082
:107C000021F324C334F023C333F022C332F021C361
:107C100031F0386A376A7E0E356E800E32AE000E55
:107C2000366EA7EC06F0E9EC07F034BE03D046EC64
:107C300008F002D048EC08F034C02AF033C029F034
:107C400032C028F031C027F0D9C232F0D8C231F0AA
:107C50003CEC08F02AC038F029C037F028C036F0D4
:107C600027C035F0A5EC06F0E9EC07F00201DA6F69
:107C700032C0DBF200010AC334F009C333F008C399
:107C800032F007C331F0386A376AC00E366E7F0EA5
:107C9000356E5FEC06F03A6E0AC334F009C333F078
:107CA00008C332F007C331F0660E386E376EE60E49
:107CB000366E810E356E23EC06F03A1607E0B60EEE
:107CC0000201D85DDA6F080ED959DB6F00010AC3D3
:107CD00034F009C333F008C332F007C331F0660E45
:107CE000386E376EE60E366E810E356E23EC06F07A
:107CF0000108D8B4ABD0266A256A800E246E7F0EA8
:107D0000236E660E2A6E296E860E286E810E276EF1
:107D10002AC034F029C033F028C032F027C031F037
:107D20000AC338F009C337F008C336F007C335F08B
:107D3000A5EC06F034C02AF033C029F032C028F098
:107D400031C027F0346A336A4C0E326E850E316EC4
:107D50002AC038F029C037F028C036F027C035F0E7
:107D60009BEC07F034C02AF033C029F032C028F071
:107D700031C027F026C038F025C037F024C036F0D7
:107D800023C035F02AC034F029C033F028C032F0C7
:107D900027C031F09BEC07F034C024F333C023F349
:107DA00032C022F331C021F3D9C232F0D8C231F04F
:107DB0003CEC08F0386AE00E376E080E366E8A0E1C
:107DC000356EA7EC06F034C026F033C025F032C083
:107DD00024F031C023F024C334F023C333F022C392
:107DE00032F021C331F0386A376A7E0E356E800E6C
:107DF00032AE000E366EA7EC06F0E9EC07F034BEAA
:107E000003D046EC08F002D048EC08F034C02AF069
:107E100033C029F032C028F031C027F026C034F03A
:107E200025C033F024C032F023C031F02AC038F02E
:107E300029C037F028C036F027C035F0A5EC06F091
:107E4000E9EC07F00201DA6F32C0DBF20001DBC2BD
:107E500032F0DAC231F03CEC08F0C8C238F0C7C2E8
:107E600037F0C6C236F0C5C235F09BEC07F09BEC8C
:107E700006F00201EF6F32C0F0F200013FEF1CF09C
:107E800081A2FED7949A8B9A020189510B6E010E42
:107E90000301586F030158510B5C000115E3820E7A
:107EA000026E400E096E810E036E010E046E0A6EA4
:107EB00002EE89F003015851EB50106E4AEC03F0CA
:107EC0000301582B0001E6E3949A8B8A12008190FB
:107ED000D7DF81A2FED7949A8B9A820E026E400E53
:107EE000096E810E036E010E046E0A6E440E106E52
:107EF0004AEC03F0820E026E800E096E810E036E54
:107F0000010E046E0A6A1EEC03F010C01CF303019C
:107F10001C29000108E0949A8B8A010E75EC03F08D
:107F2000949A8B9ADAD702EE89F003015851EB50FC
:107F30000C6E0C041C6F586B030158511C5D000142
:107F400015E3820E026E800E096E810E036E010E25
:107F5000046E0A6A1EEC03F002EE89F00301585128
:107F600010C0EBFF0301582B0001E6E3949A8B8AC3
:107F70001200010E0201896F8A6F080E8B6F0001DB
:107F8000A6DF02018B510C6E640E0C5C000102E155
:107F900003012A890201CF6B020ECE6F03012A5121
:107FA0000001E8B892D01F0E0201D35D000114E376
:107FB00011E14A0E0201D25D00010EE30BE1DD0E7C
:107FC0000201D15D000108E305E1400E0201D05D30
:107FD000000102E3000E01D0010E3A6E010E020113
:107FE000D05DB10ED159080ED259190ED3590001E6
:107FF00002E2000E01D0010E3A1605E0040E020165
:10800000CE6F020ECF6F140E0201D35D000114E398
:1080100011E1DC0E0201D25D00010EE30BE1930ED3
:108020000201D15D000108E305E1800E0201D05D8F
:10803000000102E3000E01D0010E3A6E010E0201B2
:10804000D05D7F0ED159ED0ED259100ED3590001DB
:1080500002E2000E01D0010E3A1605E0060E020102
:10806000CE6F030ECF6F0A0E0201D35D000114E341
:1080700011E16E0E0201D25D00010EE30BE1490E2B
:108080000201D15D000108E305E1C00E0201D05DEF
:10809000000102E3000E01D0010E3A6E810E0201D2
:1080A000D05DBF0ED159760ED259080ED3590001BA
:1080B00002E2000E01D0010E3A1605E00C0E02019C
:1080C000CE6F050ECF6F000151D0400E0201D05D82
:1080D000720ED159050ED2592A0ED359000105E26C
:1080E000030E0201CE6F010ECF6FC00E0201D05DF4
:1080F000EC0ED1594F0ED2591C0ED359000105E296
:10810000040E0201CE6F020ECF6F400E0201D05D51
:108110005A0ED1590A0ED259150ED359000105E253
:10812000060E0201CE6F030ECF6FC00E0201D05DAE
:10813000D90ED1593E0ED2590E0ED359000105E287
:10814000080E0201CE6F040ECF6F400E0201D05D0B
:10815000CE0ED1598C0ED2590A0ED359000105E228
:108160000C0E0201CE6F050ECF6F0001136A080ED0
:10817000126E116A106A1B6A1A6A196ACEC218F066
:108180005AEC04F013C0F4F212C0F3F211C0F2F290
:1081900010C0F1F2D7C234F0D6C233F0D5C232F0FB
:1081A000D4C231F046EC08F034C038F033C037F0B8
:1081B00032C036F031C035F0F4C234F0F3C233F0DF
:1081C000F2C232F0F1C231F046EC08F035EC07F0C3
:1081D00034C0C8F233C0C7F232C0C6F231C0C5F2F3
:1081E000D7C213F0D6C212F0D5C211F0D4C210F02B
:1081F0001B6A1A6A196ACEC218F015EC04F013C093
:10820000BFF212C0BEF211C0BDF210C0BCF2D3C2A8
:1082100013F0D2C212F0D1C211F0D0C210F0BFC21E
:108220001BF0BEC21AF0BDC219F0BCC218F015ECAA
:1082300004F013C026F012C025F011C024F010C0C5
:1082400023F023040201C06FD3C213F0D2C212F094
:10825000D1C211F0D0C210F0BFC21BF0BEC21AF0E2
:10826000BDC219F0BCC218F015EC04F030C0F4F235
:108270002FC0F3F22EC0F2F22DC0F1F2BFC234F0E3
:10828000BEC233F0BDC232F0BCC231F046EC08F0E1
:1082900034C038F033C037F032C036F031C035F07A
:1082A000F4C234F0F3C233F0F2C232F0F1C231F072
:1082B00046EC08F035EC07F034C0C4F233C0C3F22A
:1082C00032C0C2F231C0C1F2346A336A326A7F0E00
:1082D000316EC4C238F0C3C237F0C2C236F0C1C278
:1082E00035F0A7EC06F034C0C4F233C0C3F232C09C
:1082F000C2F231C0C1F2346A336A326A920E316E10
:10830000C4C238F0C3C237F0C2C236F0C1C235F0C1
:108310009BEC07F0E9EC07F0C96F32C0CAF233C03A
:10832000CBF234C0CCF2CBC2E2F2CAC2E1F2C9C293
:10833000E0F2080E896F110E8A6F400E8B6F040EEB
:108340008C6F8D6BC0C28EF2E2C28FF2E1C290F2EE
:10835000E0C291F2000140EF3FF0719E0301A56B76
:10836000A46BA36BA26BA96BA86BA76BA66BE3ECCA
:1083700002F0EE0EADEC02F0AA0EADEC02F091ECC4
:1083800002F05B6F91EC02F05A6F91EC02F05D6FBE
:1083900091EC02F05C6F91EC02F05F6F91EC02F0F7
:1083A0005E6F91EC02F0616F91EC02F0606F91EC06
:1083B00002F0636F91EC02F0626F91EC02F0656F76
:1083C0008FEC02F0646FC0EC02F0E3EC02F0EE0E12
:1083D000ADEC02F0B60EADEC02F091EC02F0676F7E
:1083E00091EC02F0666F91EC02F0696F91EC02F093
:1083F000686F91EC02F0816F91EC02F0806F91EC6C
:1084000002F0836F91EC02F0826F91EC02F0856FC5
:108410008FEC02F0846FC0EC02F0718E000112004C
:10842000719E8BD8A9C389F3A8C388F3A7C387F328
:10843000A6C386F3A5C38DF3A4C38CF3A3C38BF3A8
:10844000A2C38AF3C80E75EC03F077D8A9C395F3DD
:10845000A8C394F3A7C393F3A6C392F3A5C399F358
:10846000A4C398F3A3C397F3A2C396F3C80E75EC05
:1084700003F063D803018651A625236E8751A721F7
:10848000246E8851A821256E8951A921266E92510A
:108490002324866F93512420876F94512520886F61
:1084A00095512620896F89C313F088C312F087C3C2
:1084B00011F086C310F01B6A1A6A196A030E186E4F
:1084C00015EC04F013C0A9F312C0A8F311C0A7F370
:1084D00010C0A6F396518A25236E97518B21246EE6
:1084E00098518C21256E99518D21266EA2512324FD
:1084F0008A6FA35124208B6FA45125208C6FA55126
:1085000026208D6F8DC313F08CC312F08BC311F036
:108510008AC310F01B6A1A6A196A030E186E15ECEA
:1085200004F013C0A5F312C0A4F311C0A3F310C04C
:10853000A2F3000148D8718E1200E3EC02F0EE0EB7
:10854000ADEC02F0F40EADEC02F02E0EABEC02F04E
:10855000050E75EC03F0EE0EADEC02F0F60EADEC90
:1085600002F091EC02F00301B36F8FEC02F0B26FF6
:10857000C0EC02F0B3C3A3F3B2C3A2F3E3EC02F086
:10858000EE0EADEC02F0F40EADEC02F0340EABECFE
:1085900002F0050E75EC03F0EE0EADEC02F0F60EF7
:1085A000ADEC02F091EC02F0B46F91EC02F0B36F1D
:1085B0008FEC02F0B26FC0EC02F0B4C3A7F3B3C308
:1085C000A6F30001120003016451A25D316E6551F2
:1085D000A359326E000E65BFFF0EA459336E000E14
:1085E00065BFFF0EA559346E48EC08F034C026F084
:1085F00033C025F032C024F031C023F063C332F021
:1086000062C331F03CEC08F026C038F025C037F0EA
:1086100024C036F023C035F09BEC07F034C024F3BF
:1086200033C023F332C022F331C021F324C3BDF39E
:1086300023C3BCF322C3BBF30F0E215D02E23D84D2
:10864000000E0301BA6F83C332F082C331F03CECF9
:1086500008F034C026F033C025F032C024F031C019
:1086600023F00B0E232402E33D82FF0E0001236E54
:10867000BDC32AF0BCC329F0BBC328F0BAC327F09E
:1086800085C332F084C331F03CEC08F02AC038F0E6
:1086900029C037F028C036F027C035F0A7EC06F027
:1086A00034C02AF033C029F032C028F031C027F09E
:1086B00026C034F025C033F024C032F023C031F09E
:1086C0002AC038F029C037F028C036F027C035F06E
:1086D00035EC07F034C0C1F333C0C0F332C0BFF390
:1086E00031C0BEF3BDC338F0BCC337F0BBC336F0F6
:1086F000BAC335F0C1C334F0C0C333F0BFC332F0E6
:10870000BEC331F0A7EC06F034C0D1F333C0D0F3D0
:1087100032C0CFF331C0CEF3346A336A326A820E8C
:10872000316ED1C338F0D0C337F0CFC336F0CEC3EB
:1087300035F0A7EC06F034C026F033C025F032C087
:1087400024F031C023F0386A376A366A830E356EFA
:1087500026C034F025C033F024C032F023C031F0FD
:1087600035EC07F0E9EC07F00301AA6F32C0ABF378
:1087700033C0ACF334C0ADF3386A376A200E366EBE
:10878000820E356EADC334F0ACC333F0ABC332F000
:10879000AAC331F048EC08F035EC07F034C011F40E
:1087A00033C010F432C00FF431C00EF4386A376AA7
:1087B0007A0E366E8A0E356ED1C334F0D0C333F0E4
:1087C000CFC332F0CEC331F0A5EC06F034C0D5F300
:1087D00033C0D4F332C0D3F331C0D2F3D5C338F0B1
:1087E000D4C337F0D3C336F0D2C335F0D5C334F099
:1087F000D4C333F0D3C332F0D2C331F09BEC07F0D3
:1088000034C026F033C025F032C024F031C023F04C
:1088100026C024F325C023F324C022F30C0E235CCE
:1088200002E23D84000E0301216F69C332F068C388
:1088300031F03CEC08F024C338F023C337F022C3F6
:1088400036F021C335F09BEC07F034C0BDF333C0E4
:10885000BCF332C0BBF331C0BAF35DC332F05CC3CA
:1088600031F03CEC08F0D5C338F0D4C337F0D3C3B3
:1088700036F0D2C335F09BEC07F034C0C1F333C0FF
:10888000C0F332C0BFF331C0BEF3BDC338F0BCC3C8
:1088900037F0BBC336F0BAC335F0C1C334F0C0C340
:1088A00033F0BFC332F0BEC331F0A7EC06F034C0E2
:1088B00026F033C025F032C024F031C023F026C0AA
:1088C000C5F325C0C4F324C0C3F30B0E235C02E23E
:1088D0003D84000E0301C26F5BC332F05AC331F016
:1088E0003CEC08F034C026F033C025F032C024F050
:1088F00031C023F0020E232402E33D82FF0E00016B
:10890000236E26C038F025C037F024C036F023C0CF
:1089100035F0C5C334F0C4C333F0C3C332F0C2C3AF
:1089200031F0A7EC06F034C026F033C025F032C099
:1089300024F031C023F0346A336A326A800E316E1B
:1089400026C038F025C037F024C036F023C035F0FB
:10895000A7EC06F034C026F033C025F032C024F076
:1089600031C023F026C0C9F325C0C8F324C0C7F323
:10897000020E235C02E23D84000E0301C66F5FC35A
:1089800032F05EC331F03CEC08F0D5C338F0D4C30C
:1089900037F0D3C336F0D2C335F09BEC07F034C0C8
:1089A00026F033C025F032C024F031C023F026C0B9
:1089B000BDF325C0BCF324C0BBF30D0E235C02E263
:1089C0003D84000E0301BA6F67C332F066C331F015
:1089D0003CEC08F024C338F023C337F022C336F050
:1089E00021C335F09BEC07F034C026F033C025F0EE
:1089F00032C024F031C023F026C0C1F325C0C0F33B
:108A000024C0BFF3100E235C02E23D84000E03017C
:108A1000BE6FBDC326F0BCC325F0BBC324F0BAC3F0
:108A200023F026C038F025C037F024C036F023C02C
:108A300035F0C1C334F0C0C333F0BFC332F0BEC39E
:108A400031F0A7EC06F034C026F033C025F032C078
:108A500024F031C023F0346A336A326A800E316EFA
:108A600026C038F025C037F024C036F023C035F0DA
:108A7000A7EC06F034C026F033C025F032C024F055
:108A800031C023F026C0C5F325C0C4F324C0C3F30E
:108A9000020E235C02E23D84000E0301C26F61C33B
:108AA00032F060C331F044EC08F034C026F033C03B
:108AB00025F032C024F031C023F0C5C32AF0C4C36E
:108AC00029F0C3C328F0C2C327F0346A336A326A7C
:108AD0008E0E316E2AC038F029C037F028C036F02B
:108AE00027C035F0A7EC06F034C02AF033C029F0D7
:108AF00032C028F031C027F026C038F025C037F04A
:108B000024C036F023C035F02AC034F029C033F039
:108B100028C032F027C031F09BEC07F034C026F0BB
:108B200033C025F032C024F031C023F026C0CDF38D
:108B300025C0CCF324C0CBF30F0E235C02E23D84AE
:108B4000000E0301CA6FA9C334F0A8C333F0A7C352
:108B500032F0A6C331F048EC08F0C9C338F0C8C3FE
:108B600037F0C7C336F0C6C335F0A5EC06F034C005
:108B700026F033C025F032C024F031C023F0346A2F
:108B8000500E336E430E326E8E0E316E26C038F0AC
:108B900025C037F024C036F023C035F09BEC07F039
:108BA000E9EC07F07A6F32C07BF333C07CF334C05A
:108BB0007DF37DC334F07CC333F07BC332F07AC3E2
:108BC00031F048EC08F0386A376A366A800E356E44
:108BD0009BEC07F034C026F033C025F032C024F0FF
:108BE00031C023F026C034F025C033F024C032F069
:108BF00023C031F0CDC338F0CCC337F0CBC336F04F
:108C0000CAC335F035EC07F034C0D9F333C0D8F31C
:108C100032C0D7F331C0D6F3D9C324F3D8C323F37A
:108C2000D7C322F3080ED65D02E23D84000E030195
:108C3000216F24C338F023C337F022C336F021C399
:108C400035F024C334F023C333F022C332F021C300
:108C500031F09BEC07F034C0BDF333C0BCF332C03D
:108C6000BBF331C0BAF3346AE00E336E3D0E326EA0
:108C70008A0E316EBDC338F0BCC337F0BBC336F0CB
:108C8000BAC335F09BEC07F034C026F033C025F0B2
:108C900032C024F031C023F026C0BDF325C0BCF3A0
:108CA00024C0BBF3100E235C02E23D84000E0301DE
:108CB000BA6F346AE80E336EE50E326E8B0E316E8B
:108CC000D9C338F0D8C337F0D7C336F0D6C335F0A0
:108CD0009BEC07F034C026F033C025F032C024F0FE
:108CE00031C023F026C0C1F325C0C0F324C0BFF3B8
:108CF000100E235C02E23D84000E0301BE6FD9C357
:108D000026F0D8C325F0D7C324F0D6C323F0BDC3C3
:108D10002AF0BCC329F0BBC328F0BAC327F02AC08D
:108D200038F029C037F028C036F027C035F0C1C36D
:108D300034F0C0C333F0BFC332F0BEC331F0A7EC90
:108D400006F034C02AF033C029F032C028F031C018
:108D500027F0346AF00E336E6C0E326E8A0E316E6E
:108D60002AC038F029C037F028C036F027C035F0C7
:108D7000A7EC06F034C02AF033C029F032C028F046
:108D800031C027F0040E275E02E23D84276A00010D
:108D900026C038F025C037F024C036F023C035F0A7
:108DA0002AC034F029C033F028C032F027C031F097
:108DB000A7EC06F0E9EC07F00301AE6F32C0AFF3A9
:108DC00033C0B0F334C0B1F3386A376A480E366E38
:108DD000850E356EB1C334F0B0C333F0AFC332F09B
:108DE000AEC331F048EC08F035EC07F034C026F0A3
:108DF00033C025F032C024F031C023F09A0E346E17
:108E0000990E336E2D0E326E830E316E26C038F001
:108E100025C037F024C036F023C035F0A7EC06F0AB
:108E200034C0D9F333C0D8F332C0D7F331C0D6F34E
:108E300000011200B50E0201896F620E8A6F060EE4
:108E40008B6F240E8C6F8D6F8E6B8F699069080EFF
:108E5000916F030E926F936B946B956B966B100EE4
:108E6000976F270E986F996B9A6B050E9B6F9C6B93
:108E7000FA0E9D6F9E6B9F6FA06B640EA16FA26B2D
:108E80002C0EA36F010EA46FA56BA66BA76BA86B2E
:108E9000A96BAA6BAB6BAC6BAD6BAE6BAF6BB06B16
:108EA000B16BB26B160EB36FDC0EB46FB36BB46BF9
:108EB000020EC06F2A0E0201C05D000118E202011D
:108EC000B3510E6E02EE89F0C051EB500F6E0E24BE
:108ED0000C6E0CC0B3F2B4510E6EB3510F6E0E2473
:108EE0000C6E0CC0B4F20201C02B0001E3E30201DE
:108EF000C06B2C0E0201C05D00010BE202EE89F096
:108F00000201C051EB5032EC02F00201C02B000113
:108F1000F0E38BC20CF00CC08FF28CC20CF00CC0D2
:108F200090F2B50E0201896F620E8A6F050E8B6F8B
:108F3000010E8C6F020E8D6F8E6B916B926B020E19
:108F4000C06F080E0201C05D000118E202019151DC
:108F50000E6E02EE89F0C051EB500F6E0E240C6EB7
:108F60000CC091F292510E6E91510F6E0E240C6E48
:108F70000CC092F20201C02B0001E3E30B0E096E5C
:108F8000B80E026E0DEC02F039E303011C6F020112
:108F900089510C6E03011C510C5C00010BE00B0E9F
:108FA000096EB80E026E0DEC02F028E303011C6F8F
:108FB0000001EDD7010E0201C06F080E0201C05D75
:108FC000000118E20B0E096EB80E026E0DEC02F0F5
:108FD00015E303011C6F02EE89F00201C051EB5052
:108FE0000C6E03011C510C5C000108E10201C02B56
:108FF0000001E3E303012A950001120003012A8521
:0C900000000112000400FED70400FED79F
:020000040030CA
:03000100C80E33F3
:020005003D803C
:0600080008C00FE00F40EC
:0200000400F00A
:100000004243303453FFFFFFFFFFFFFFFFFFFFFFBF
:100010004243504C342E35FFFFFFFFFFFFFFFFFF31
:10002000343334383030303030FFFFFFFFFFFFFF14
:10003000383730FFFFFFFFFFFFFFFFFFFFFFFFFF2E
:10004000313030FFFFFFFFFFFFFFFFFFFFFFFFFF2C
:100050003732FFFFFFFFFFFFFFFFFFFFFFFFFFFF45
:1000600031FFFFFFFFFFFFFFFFFFFFFFFFFFFFFF6E
:100070003530FFFFFFFFFFFFFFFFFFFFFFFFFFFF29
:1000800069090606F82401B004544400FFFFFFFF8D
:100090006A293F3E3C3830202123272F4755013124
:1000A0000611150902140B10041E0D1207050F1678
:0A00B0001B0A08030C180E191D139B
:00000001FF
